:10000000081C0020111C0000651C0000A91A00003B
:10001000A91A0000A91A0000A91A0000A91A0000D4
:10002000A91A0000A91A0000A91A0000B1160000C0
:10003000A91A0000A91A00006D160000A91A0000F4
:10004000D51B00000B800000D51B0000D51B000055
:10005000D51B0000D51B0000D51B0000D51B0000E0
:10006000D51B0000D51B0000D51B0000D51B0000D0
:10007000D51B0000D51B0000D51B0000D51B0000C0
:10008000D51B0000D51B0000D51B0000D51B0000B0
:10009000D51B0000D51B0000D51B0000D51B0000A0
:1000A000D51B0000D51B0000D51B0000D51B000090
:1000B000D51B0000D51B0000D51B0000D51B000080
:1000C000D51B0000D51B0000D51B0000D51B000070
:1000D000D51B0000D51B0000D51B0000D51B000060
:1000E000D51B0000D51B0000D51B0000D51B000050
:1000F000D51B0000D51B0000D51B0000D51B000040
:1001000000000000D512000000000000211A0000CD
:10011000D82B0020F19A000000000000211A0000F6
:1001200000000000211A000000000000211A000059
:10013000000000008993000000000000211A000068
:1001400000000000211A000000000000211A000039
:1001500000000000211A000000000000D17F000014
:1001600000000000211A0000E42B0020599E00002E
:1001700000000000211A000000000000211A000009
:1001800000000000211A000000000000D11400004F
:1001900000000000211A000000000000211A0000E9
:1001A00000000000211A000000000000211A0000D9
:1001B00000000000211A000000000000211A0000C9
:1001C000000000000580000000000000211A00006F
:1001D00000000000211A000000000000211A0000A9
:1001E00000000000211A000000000000211A000099
:1001F00000000000211A000000000000211A000089
:1002000000000000211A000000000000211A000078
:1002100000000000211A000000000000211A000068
:1002200000000000211A000000000000211A000058
:1002300000000000211A000000000000211A000048
:1002400000000000211A000000000000211A000038
:1002500000000000211A000000000000211A000028
:1002600000000000211A000000000000211A000018
:1002700000000000211A000000000000211A000008
:1002800053B94AB9002908BF00281CBF4FF0FF31FD
:100290004FF0FF3000F086B9ADF1080C6DE904CEE7
:1002A00000F01AF8DDF804E0DDE9022304B070473D
:1002B000430803F05533C01A830803F0333300F0CA
:1002C0003330184400EB101000F00F3000EB00202A
:1002D00000EB0040000E70472DE9F047089E0446F1
:1002E0008846002B4BD18A42154667D9B2FA82F272
:1002F0004AB1C2F1200701FA02F320FA07F795404C
:1003000047EA030894404FEA154E230CB8FBFEF76A
:100310001FFA85FC0EFB178843EA084307FB0CF124
:10032000994209D9EB1807F1FF3080F01B819942FF
:1003300040F21881023F2B445B1AA4B2B3FBFEF0DB
:100340000EFB103344EA034400FB0CFCA44509D91E
:100350002C1900F1FF3380F00781A44540F204819D
:1003600002382C4440EA0740A4EB0C0400271EB1DD
:10037000D4400023C6E900433946BDE8F0878B42EC
:1003800009D9002E00F0EB800027C6E900013846AD
:100390003946BDE8F087B3FA83F7002F47D18B4287
:1003A00002D3824200F2FA80841A61EB0303012037
:1003B0009846002EE0D0C6E90048DDE702B9FFDE2E
:1003C000B2FA82F2002A40F08F80491B4FEA154EA4
:1003D0001FFA85F80127B1FBFEFC230C0EFB1C1154
:1003E00043EA014308FB0CF1994207D9EB180CF1E1
:1003F000FF3002D2994200F2CD808446591AA3B24E
:10040000B1FBFEF00EFB101443EA044408FB00F8B5
:10041000A04507D92C1900F1FF3302D2A04500F204
:10042000B6801846A4EB080440EA0C409FE7C7F1E9
:10043000200CBB4022FA0CFE4EEA030E01FA07F430
:1004400020FA0CF521FA0CF34FEA1E482543B3FBC2
:10045000F8F92C0C08FB19331FFA8EFA44EA03430F
:1004600009FB0AF49C4202FA07F200FA07F10BD9E1
:100470001EEB030309F1FF3080F087809C4240F2BD
:100480008480A9F1020973441B1BADB2B3FBF8F0E1
:1004900008FB103345EA034400FB0AFAA24508D9D9
:1004A0001EEB040400F1FF336BD2A24569D9023878
:1004B000744440EA0940A0FB0289A4EB0A044C45BD
:1004C000C2464B4654D351D0002E69D0B1EB0A0539
:1004D00064EB030404FA0CFCFD40FC404CEA050507
:1004E000C6E90054002747E7C2F1200320FA03F7CA
:1004F000954001FA02F021FA03F34FEA154E384312
:10050000010CB3FBFEF71FFA85F80EFB173341EA27
:10051000034107FB08F38B4204FA02F407D9691878
:1005200007F1FF3C2FD28B422DD9023F2944CB1A31
:1005300081B2B3FBFEF00EFB103341EA034100FB36
:1005400008F38B4207D9691800F1FF3C17D28B42A0
:1005500015D902382944C91A40EA07473BE737460C
:10056000304609E70746E7E61846FBE64145ABD2C9
:10057000B8EB020A69EB0E0201381346A4E76046A5
:10058000E9E7184695E76746D1E781467CE70238F8
:100590002C4447E7ACF1020C2B442FE7384608E720
:1005A0003746E9E6704700BF436810B45C681346FD
:1005B000A4460A4610BC00216047436810B41C687A
:1005C0000A46A4460123002110BC604703689B68CB
:1005D00001F5E0711B68022243F8212070470000FA
:1005E00010B55B4C02212068FFF7F0FF2068042162
:1005F000FFF7ECFF20680621FFF7E8FF20680821DD
:10060000FFF7E4FF20680821FFF7E0FF20680821DA
:10061000FFF7DCFF20680821FFF7D8FF20680821DA
:10062000FFF7D4FF20680821FFF7D0FF20680B21D7
:10063000FFF7CCFF0C212068FFF7BFFF01220C2140
:100640002068FFF7B1FF20680D21FFF7BFFF20688A
:100650000E21FFF7BBFF20680F21FFF7B7FF2068CF
:100660001021FFF7B3FF20681121FFF7AFFF2068CB
:100670001421FFF7ABFF20681521FFF7A7FF2068C3
:100680001621FFF7A3FF20681721FFF79FFF2068BF
:100690001821FFF79BFF20681921FFF797FF2068BB
:1006A0001A21FFF793FF20681B21FFF78FFF2068B7
:1006B0001C21FFF78BFF20681D21FFF787FF2068B3
:1006C0001E21FFF783FF2068224C1F21FFF77EFFCA
:1006D00020680121FFF77AFF20680221FFF776FFEB
:1006E00020680321FFF772FF20680421FFF76EFFE7
:1006F00020680521FFF76AFF20680621FFF766FFE3
:1007000020680721FFF762FF20680921FFF75EFFDD
:1007100020680A21FFF75AFF20680B21FFF756FFD8
:100720000C212068FFF749FF01220C212068FFF708
:100730003BFF20680D21FFF749FF20680E21FFF7DE
:1007400045FF20680F21BDE81040FFF73FBF00BF05
:10075000A80E0020AC0E002038B50D480D4D09F054
:10076000EDFB0D4B18600D4809F0E8FB0C4B1860D1
:100770000C4809F0E3FBFFF733FF0A2442F2107044
:100780000AF0AEF82146284600F0A6FB0A34F5E749
:10079000D9B10000EEB10000A80E0020E0B10000C9
:1007A000AC0E0020E7B1000010B54FF02003EFF3CE
:1007B000118483F3118800F0CBFB084A0123C2F8AF
:1007C00040354FF08042C2F87835054B4FF0FF328C
:1007D0009A62DA6284F31188002010BD00E00140C3
:1007E00000ED00E008B50446084611461A46A04749
:1007F0000AF0A2F801F0C8F970B5C668C07A0C25F5
:100800004D43884206EB0504B4BF715921462024AC
:1008100092FBF4F401EB8401196002F01F0070BD3B
:1008200007B501ABFFF7E8FF019A012303FA00F0D7
:1008300013680343136003B05DF804FB07B501AB15
:10084000FFF7DAFF019A012303FA00F0136823EAA5
:100850000003136003B05DF804FB2DE9F843044680
:1008600043680589006894F80AC05D432844002164
:100870004FF00C0E8C4505DC00252389AB4222DCB1
:10088000BDE8F883D4F80C80B5FBF3F20EFB01F75A
:100890001F2A08EB0706C8BF1F324FEA930306F171
:1008A0000409C8BF520903F10303C6E9019923F003
:1008B0000303D4BFE17248F8070001F10101C8BF8A
:1008C00000EB8200D6E76268E36820686A4381181B
:1008D0001E1D86509A684A609A6820461160996089
:1008E0002A460021FFF79CFF0135C6E72DE9F04FAE
:1008F00089B0867A00AFC7E90132B3000A3303F446
:10090000FF63ADEB030D4368E94603334A4623F02A
:10091000030342F8043905464FF0FF3400234FF03B
:100920000C0C581E9E42F86109DD2BB1106880083E
:10093000033020F003005060506888420BD2FB69FE
:10094000013314D1BA6C002313606FF00B0024370D
:10095000BD46BDE8F08FE8680CFB030000F1040E13
:1009600040680432704518BF1C460133D9E7631C48
:10097000E8D0E96859F824200C2303FB041353F84A
:10098000046F9E4263D0D6E90013196031684B6052
:100990002B682146F31A284693FBF2F2FFF74EFF2D
:1009A000A9EB890304F1010B3B6109EB8404F969AC
:1009B0002B680BF1FF329142A6EB03030DDCBA6802
:1009C0001146FA690A6059F8222093FBF2F37A681B
:1009D0001360BB6C00201E60B9E754F8042B93FB36
:1009E000F2F33A699B00FB6004EB440313447B6120
:1009F0004FF0010AD4F800800AFB08F3BB61F3183A
:100A00003B60FB6859460AEB03022846FFF708FFE4
:100A10003B682A68298908F1FF389844A8EB020846
:100A20006A684A4390450AD2EA687969B8690A4413
:100A3000111D31509168596091680B6093600AF103
:100A4000010ABAF1040FD5D10BF1010BAFE76FF03A
:100A50000A007CE72DE9F04F85B0837A9B000A33CA
:100A600003F4FF6300AFADEB030D4368EA460333C5
:100A700023F003030546CAF80030544601208142A2
:100A80004CD20C4616463246214628465AF8248057
:100A9000D5F80090FFF7C4FE002C48D007F10C03F6
:100AA000324621462846FFF7A7FEFA68042390FB4A
:100AB000F3F083001068D84000F00F000F2836D103
:100AC00026F003034FF000097B6008F1FF3B7B68D1
:100AD0004B441A46214628463B60FFF7AFFE3B6871
:100AE0009E4212D008FB03F2B5F808E06B68296853
:100AF00002EB0B0C03FB0EF39C4501EB020004D24E
:100B000040688B5803608B58586009F10109B9F1AE
:100B1000040FDCD196FBF9F6013CB4E723689B088F
:100B2000033323F0030344F8043F0130A7E708FB35
:100B300006F62A68696809EB060308F1FF3898444D
:100B4000A8EB02082A89514388450BD2E9680C2298
:100B500002FB0414221D49F80620A2685A60A2680C
:100B60001360A3601437BD46BDE8F08F00207047C6
:100B70000B6801330B60014B1B6818476829002084
:100B80002DE9F04F85B09B460E9CDFF890A0012C1C
:100B9000B8BF0124012B0CBF30232023154680460B
:100BA00089460194029301260A2700220AF10104D2
:100BB0000AB9AA451FD2B5FBF4F049463030C04708
:100BC00001360122013F012FB5FBF4F14FF00A037A
:100BD00004FB1155BAFBF3FAE8D1494605F13000A0
:100BE000C047BBF1030F03D1019B9C1B002C0FDC02
:100BF00005B0BDE8F08F019BBB42E3DBBBF1020F08
:100C0000E0D84946029803920136C047039AD9E7D3
:100C100049462020C047013CE8E700BFFFC99A3B96
:100C200030B58A680C68551C14B14B68934201DCDE
:100C30008D6030BD013B934208BF00228D600CBF28
:100C4000E254A054F5E70000014B1860704700BF64
:100C5000682900202DE9F04F89B01C464FF0000AAA
:100C6000531E06460F4604934FF0FF39D046002529
:100C700005E06DB9252800F012813946B047049B84
:100C800013F8010F04930028F3D109B0BDE8F08FE9
:100C9000642861D019D839280AD8312850D22D2893
:100CA0003CD030283DD0252808D13946B047DEE772
:100CB000582800F08880632800F0EB803946252012
:100CC000B047049B39461878F0E7702871D006D8F1
:100CD000692841D06C283CD06828D0D0EEE7752830
:100CE00057D017D87328E9D1236804F1040B1C46A8
:100CF000254615F8010B002840F0C080B8F1030F1D
:100D000040F0D680E41AA9EB0404002C00F3BC8068
:100D10005C46ACE7782856D07A28DEE74FF0030827
:100D2000ADE7B9F1000F0EDAB8F1000F00F0BD80A9
:100D3000A0F13009B8F1000F08BF4FF002089EE79C
:100D4000B9F1000FF4DB0A2303FB0909A9F130090B
:100D5000F0E70AF1010A92E7BAF1010FC5BF0734C3
:100D600024F0070325681D68D4BF043403F1080488
:100D7000002D05DA39462D20B0476D4209F1FF39C3
:100D8000CDF8009043462A4639463046FFF7F8FE34
:100D90006DE7BAF1010FC5BF073424F007032268DD
:100DA0001A68CDF80090CCBF03F108040434434620
:100DB000EAE739463020B04739467820B0474FF04F
:100DC00008094FF00108BAF1010FC7BF073424F03A
:100DD000070323680593C2BF03F108041B6805934A
:100DE0004FF008024FF00003D8BF04340393079379
:100DF00093460BF1FF3B059B4FEA8B0023FA00F073
:100E000010F00F0009D1079B13B9BBF1000F24D1DB
:100E10004FF0300C07E0069AEBE709288CBF4FF043
:100E2000570C4FF0300C394660440692B047039B94
:100E3000079501330393BBF1000FECD1B8F1030F19
:100E40007FF415AF039BC3EB4905002D7FF70FAF70
:100E500039462020B047013DF7E7531E91450693E0
:100E6000E9DBB8F1010F03D139463020B047E2E7A2
:100E7000B8F1020FDFD139462020F7E73946039356
:100E80002C46B047039B33E739462020B047013C4E
:100E90003BE72068251D3946B0472C46E7E6AA46C1
:100EA000A8464FF0FF390125E9E64FF00108E6E6D4
:100EB0005C460546E3E6000013B502AC002344F8A7
:100EC000043D02460B4603482146FFF7C3FE019846
:100ED00002B010BD710B00000FB407B504A951F8A2
:100EE000040B0191FFF7E8FF03B05DF804EB04B0D9
:100EF000704700000CB430B585B008ABCDE90101F6
:100F000053F8042B00930446002501A906480395D5
:100F1000FFF7A0FEDDE902309842B8BF255405B0C6
:100F2000BDE8304002B07047210C0000704700005F
:100F3000054B1B68082B01BF044B1868B0FA80F002
:100F4000400918BF00207047300100103401001024
:100F500008B54FF080430022C3F80C21C3F81021DC
:100F6000C3F838254FF0805203F54043D2F80414FB
:100F7000C3F82015D2F80814C3F82415D2F80C14BD
:100F8000C3F82815D2F81014C3F82C15D2F814148D
:100F9000C3F83015D2F81814C3F83415D2F81C145D
:100FA000C3F84015D2F82014C3F84415D2F824141D
:100FB000C3F84815D2F82814C3F84C15D2F82C14ED
:100FC000C3F85015D2F83014C3F85415D2F83414BD
:100FD000C3F86015D2F83814C3F86415D2F83C147D
:100FE000C3F86815D2F84014C3F86C15D2F844243D
:100FF000C3F87025FFF79CFF10B1334B334A1A60DA
:10100000FFF796FF18B1324BFB22C3F81825FFF704
:101010008FFF48B12F49304B0A681B6822F00F023E
:1010200003F00F0313430B60FFF782FF18B12B4B44
:101030004FF400721A604FF08043D3F80024D207B7
:1010400044BF6FF00102C3F800244FF01023D3F81F
:101050000022002A03DBD3F80432002B2FDA204BC6
:101060000122C3F80425D3F80024002AFBD04FF056
:1010700010221221C2F80012D3F80024002AFBD05B
:101080004FF010231222C3F80422154B1A46D3F84E
:1010900000140029FBD00021C3F80415D2F8003455
:1010A000002BFBD0BFF34F8F0E490F4BCA6802F4E1
:1010B000E0621343CB60BFF34F8F00BFFDE70B4BE4
:1010C0000B4A1A6008BD00BF8C56004048810300DF
:1010D00000F00040E40E004058020010409602402C
:1010E00000E0014000ED00E00400FA056C2900205A
:1010F0000090D00313B5114CBFF35B8F2068BFF392
:101100005B8F60B90E4808F019FFBFF35B8F54E89E
:10111000003F44E80002002AF9D1BFF35B8F436827
:1011200004221B680DEB02019847002802DA00F048
:1011300049FA0190019802B010BD00BF00000020E4
:1011400044B2000043685B68184700207047000005
:101150000A4B70B5C6B204461B6830469847012852
:101160000AD00A2C064D03D10D212868FFF7EAFFAB
:1011700031462868FFF7E6FF204670BD7029002041
:10118000040000200148FFF75FBD00BF51110000BF
:1011900008B5044808F0D2FE034B1860FFF7F2FFD1
:1011A000002008BDE7B100000400002010B54FF09A
:1011B0002003EFF3118283F31188114C237823B9B4
:1011C00082F311886FF0440010BD013BDBB2237045
:1011D00023B182F311886FF00F00F5E7094B1878FF
:1011E000012128B1217082F311886FF00A00EBE72A
:1011F000197082F31188044A11601870E4E700BF87
:101200000A000020090000200400004008B5002268
:101210001046012100F0ECFB002000F0B7FB00209D
:1012200008BD0000F8B54FF02002EFF3118382F300
:101230001188254A1078441C147060B183F311881A
:101240004FF08043D3F80C3413F4803F14BF0020D8
:101250006FF0430007E01D4D2F782FB1107083F31E
:1012600011886FF00A00F8BD01262E7083F31188F3
:101270004FF0804419B3384600F098FBC4F8007171
:10128000D4F80433C4F804632660D4F8002192B182
:101290000022C4F800210E4A13F0010F4FF00103A1
:1012A00008BFC4F808330020C2F8803100F06EFB9C
:1012B00000232B70C4E720BF40BF20BFE5E7C4F880
:1012C00000112660F4E700BF0A000020090000209A
:1012D00000E100E0F8B54FF080430546D3F808C1BF
:1012E000D3F80423D3F80C44D3F80071D3F80401E5
:1012F000D3F80C11D3F8106102F00102BCF1000F19
:1013000003D04FF0000CC3F808C127B14FF0804361
:101310000027C3F800713AB1E30341BF4FF08043A7
:101320000122C3F808231A6120B14FF08043002244
:10133000C3F8042149B14FF080440021C4F80C11D6
:101340002846FFF733FF0123636176B14FF08043F6
:1013500000210124C3F810112846C3F80443FFF705
:1013600061FF10B9014BC3F80041F8BD00E100E096
:10137000F8B506460C464FF02002EFF3118382F3D6
:1013800011882D4A157865B183F311884FF0804399
:10139000D3F8183413F4803F0CBF6FF043000020E3
:1013A000F8BD0127177083F31188284600F0FEFA74
:1013B0004FF080430221C3F80451D3F80423C3F84B
:1013C00004131E49C3F818450F60D3F8041171B314
:1013D00092071B4F58BF02224FF000014FF001054A
:1013E000C3F804114FF0000058BFC3F80823C7F832
:1013F000805100F0CBFA4FF0804300211822C3F84F
:101400000823C3F80C11C3F8101114F00301BDD167
:101410001020C3F83805C3F804233046C3F804533A
:10142000FFF700FF0028B1D1C7F80051AEE720BF99
:1014300040BF20BFC9E700BF0800002008000040EF
:1014400000E100E0084BC3F84005D3F80435C01AAA
:1014500020F07F40054B0238984282BF044B4FF486
:101460000032C3F80021704700100140FDFF7F00EB
:1014700000E100E038B5114B114CD3F804052268A7
:10148000104D801A2B6820F07F4083420FD8B0FBAC
:10149000F3F00D490968884228BF084600FB032382
:1014A00023F07F432360094B186009F0AFFA2068EE
:1014B0002B681844BDE83840FFF7C4BF0010014056
:1014C00010000020982B00200C000020942B0020FE
:1014D000024B0022C3F84021FFF7CCBF00100140AF
:1014E000084B00281A68084B93FBF2F302DB834297
:1014F000A8BF034605490B600549086802FB0300C5
:10150000FFF7A0BF982B0020FFFF7F000C000020FA
:101510001000002008B5074B0022C3F84021064BFD
:101520004FF40032C3F88021FFF7A4FF034B0122E0
:101530001A6008BD0010014000E100E00C0000202E
:1015400070B5194808F0FAFC50B34368174D1B6892
:1015500001219847164B00241C60164B01261E6083
:10156000154BC5F808451B68C5F840354FF4803366
:10157000C5F84433C5F80433104BC5F840414FF467
:101580000032C3F8802131462246112000F030FAA3
:10159000112000F0FBF90A4B20461E602E6070BD42
:1015A0004FF0FF30FBE700BF68B2000000100140C1
:1015B000100000200C000020982B002000E100E02B
:1015C000081001400A4A0B49D2F8043570B50D687D
:1015D000094ED6E90001D2F80445A34205D168437B
:1015E0001B1A23F07F43184470BD2346F1E700BF68
:1015F00000100140982B0020C80F00200748816888
:10160000006A884208D000B509F01CF95DF804EBC7
:1016100003494FF080520A6070470000940F002089
:1016200004ED00E0044800232021C2180133302BD0
:1016300082F80013F9D1704700E100E0084A094937
:1016400093680968D966084998664B6843F08053E7
:101650004B60002383F311889368D86E704700BFF6
:10166000940F002074B8000000ED00E0202080F30B
:1016700011880D498A684FF02C001044EFF3098C53
:1016800080E8F01F094F4FF000660A6A8A603E60EA
:10169000906E0023936680F3118802F12C0090E88D
:1016A000F01F8CF309887047940F002004ED00E0D0
:1016B0001EF0040F0CBFEFF30880EFF3098081697F
:1016C00031F8021C11F0FF010229FFD000B500F033
:1016D0002BFA00BD10B5044609F02EF92268014628
:1016E000BDE810400148FFF7F7BB00BFC1B30000E1
:1016F00038B504461A480D46FFF7EEFB04F1180012
:10170000184CFFF7E7FFA36AD90602D51648FFF782
:10171000E3FBA36A1A0702D51448FFF7DDFBA36AAF
:101720009B070ED51248FFF7D7FB616BA36A18061B
:1017300007D51048FFF7D0FB1DB1A36A23F0800343
:10174000A362084CA26AD20702D50B48FFF7C4FB7C
:10175000A36A9B0602D50948FFF7BEFB002038BDEF
:101760000BB4000000ED00E022B4000034B400002F
:1017700048B4000061B4000072B4000092B40000EC
:1017800010B504461A48FFF7A7FB04F11800194CDE
:10179000FFF7A0FFA36A9A0102D51748FFF79CFB49
:1017A000A36ADB0102D51548FFF796FBA36A18036D
:1017B00002D51348FFF790FB0E4CA36A590302D5DC
:1017C0001048FFF789FBA36A9A0302D50E48FFF77A
:1017D00083FBA36ADB0302D50C48FFF77DFB054AB8
:1017E000936A6FEA03436FEA13439362002010BDCC
:1017F000C2B4000000ED00E0DBB40000EFB4000074
:101800000AB5000029B500004FB500006AB5000018
:1018100038B504461D480D46FFF75EFB04F118007D
:101820001B4CFFF757FFA36AD80404D51948BDE83D
:101830003840FFF751BBA36A190501D51648F6E7F2
:10184000A36A9A0514D51548FFF746FBA16BA36A56
:101850001B0407D51248FFF73FFB1DB1A36A23F411
:101860000043A3620A4B9B6A58050ED50D48DEE77C
:10187000A36A5905FAD4A36ADA0501D50A48D6E75E
:10188000A36A9B0401D50948D1E738BD88B200009E
:1018900000ED00E022B4000034B400009FB200006C
:1018A00061B40000B9B20000D5B2000092B40000EB
:1018B00038B5274C6368C3F30803DA1E0546092AC6
:1018C0003BD8DFE802F0053436303A3A3A3A3A3853
:1018D0002048FFF701FBE36A9A0703D51E48FFF78C
:1018E000FBFA02E0E36A5B0001D4002009E01B4838
:1018F000FFF7F2FA1A4B1B7843B101212846FFF794
:10190000F7FE2946BDE8384000F012B9154B1B78A8
:1019100023B101212846FFF77BFFE6E7124B1B8826
:101920009BB2002BE1D02846FFF72AFFE9E7002110
:10193000E4E70021EEE70D48D1E70D480D49A3F19A
:1019400010020F2BD8BF01460B48FFF7C5FACCE7B2
:1019500000ED00E01CB3000034B3000056B30000FB
:1019600028ED00E029ED00E02AED00E076B300006C
:10197000EEB2000003B30000ADB30000024A5369A9
:1019800043F010035361704700ED00E043B2002BB9
:1019900008DB012200F01F0002FA00F05B09024A96
:1019A00042F82300704700BF00E100E043B2002B83
:1019B0000DDB01225B0900F01F0002FA00F020336A
:1019C000034A42F82300BFF34F8FBFF36F8F704776
:1019D00000E100E04209054B00F01F0053F822200F
:1019E000012303FA00F01040704700BF00E100E05F
:1019F00043B2002BA8BF03F1604301F101014FEA9C
:101A00004111AEBF03F5614300F00F00034BC9B2B3
:101A1000ACBF83F800131954704700BF14ED00E009
:101A200000F042B808B572B6044BD86918B100226C
:101A3000DA6108F0A9FA62B608BD00BF940F002071
:101A4000F8B50C4616461F4604220A9B099905461E
:101A500009F0F2F9A6F1200121440C4A21F0070116
:101A6000002322F00102C5E91433C5E917468A6153
:101A7000069A4A60079A8A60089ACA604FF0807294
:101A80000F60CA61E964AB66F8BD00BFE5070000FE
:101A9000014910220A60704710ED00E0404080F3D9
:101AA000118830BF704700BF404080F31188DFF8D5
:101AB0001CC0DCF800C01CF4006C0CBFEFF3088005
:101AC000EFF3098000B5FFF7F3FE00BD04ED00E081
:101AD000042838B504460D4613D0052813D0032832
:101AE00013D10C48FFF7F8F908F026FFAA69014660
:101AF0000948FFF7F1F929462046BDE8384000F0D3
:101B000017B80648EEE70648ECE701460548FFF738
:101B1000E3F9E9E796B5000014B60000BCB5000093
:101B2000D6B50000F1B5000001460068FFF7D0BF50
:101B3000052810B50CD009F0ADF860B109F0AAF88D
:101B40000C490D4B002808BF19460C48FFF7C4F993
:101B5000FFF7A4FFFCE709F0ADF80028EED1084C30
:101B60000848A168FFF7B8F9A068BDE8104000F088
:101B70000BB800BF50B6000054B6000065B60000B8
:101B8000940F002085B6000038B505464FF02003BD
:101B9000EFF3118483F3118809F0E4F80B4B9B6891
:101BA000AB420DD10A4B5A68C2F3080222B908F0C1
:101BB00049FE2046FFF742FD5A6842F080525A60C3
:101BC0002046BDE8384008F0F7BC00BF940F002065
:101BD00000ED00E000B572B60B4AD06900281EBFC8
:101BE0000021D16108F0D0F962B6EFF30580A0F1D1
:101BF00010004FEAC0000549014409C998475DF843
:101C000004EBFFF7FBBC0000940F00200001000074
:101C1000202080F3118806484FF40061401880F3BB
:101C20000988022080F31488BFF36F8F00F006B894
:101C3000481D002030BFFFF7FDBF00BF08B5074BB0
:101C4000074A23F07F039360BFF34F8FBFF36F8F7B
:101C500008F0CAF908F0D2F908F0F4F90000000021
:101C600000ED00E008B5FFF7E5FFBDE80840FFF72D
:101C7000C5BC0000124930B50D68082D0DD8114AB9
:101C80004868002353609D4200F10C0007D10523F2
:101C90005360BFF34F8FBFF36F8F002030BD50F8FC
:101CA0000C1C50F8044C936021F01F0141F010010E
:101CB000194344F00104D16001331461E3E700BF2C
:101CC0004829002090ED00E00139034611F8012F6A
:101CD0000AB91A70704703F8012BF7E70138013988
:101CE00010F8013F11F8012F934202D1002BF7D1D8
:101CF0001A46981A704710B55AB10139841810F86D
:101D0000012B11F8013FA04201D09A42F7D0D01A1E
:101D100010BD1046FCE7F0B581EA0004A5070346B4
:101D20000BD0013B0A4491421DD1F0BD002AFCD0EA
:101D300011F8014B03F8014B013A9C07F6D11D1F26
:101D40000C468F183E1B032E08D894086FF003052D
:101D500005FB0422A40023442144E2E754F8046B69
:101D600045F8046FEEE711F8014B03F8014FDAE78D
:101D7000F0B5C9B203469C070FD141EA012444EAF9
:101D800004441D469F187E1B032E0CD8940803EBB9
:101D9000840413449C4209D1F0BD002AFCD003F80E
:101DA000011B013AE7E745F8044BECE704F8011B97
:101DB000F0E7BFF35B8F50E8003F43EA010240E8E1
:101DC000002CBCF1000FF6D1BFF35B8F18467047B3
:101DD000BFF35B8F50E8003F03EA010240E8002CAC
:101DE000BCF1000FF6D1BFF35B8F184670470000BF
:101DF00070B5064688790D4607F072F90E4B83429E
:101E000019D1284607F072F9284607F06FF90B4CF4
:101E100004EBC000436873B1284607F067F904F883
:101E20003060284607F062F904EBC000BDE870405E
:101E3000406808F090BD70BD842C00201400002084
:101E4000054BBFF35B8F1B6FBFF35B8F43FA00F053
:101E500000F00100704700BF782900202DE9F0470D
:101E6000804689461348144D4FF0FF3107F0CCF9F6
:101E7000044600F1080600213046002707F0CAF9A1
:101E80002775204607F032F905EBC000A0F8028064
:101E9000204607F02BF905EBC000032147603046D0
:101EA00007F0FCF980F80290A0F800802046BDE819
:101EB000F08700BF842C00201400002070B5154668
:101EC00086B00C4619B9FFF7C9FF044668B3012272
:101ED0000021684608F036FD204607F007F9144E49
:101EE00006EBC000C0F804D0204607F0D3F9214625
:101EF000104807F093F942F21071684608F052FD5D
:101F0000204607F0F3F816F8300030B1204607F00D
:101F100093F96FF0040006B070BD0DB12C60FAE7C4
:101F2000204607F089F92846F5E76FF03600F2E71A
:101F3000140000201C2A002038B50221054642F278
:101F40000C00FFF78BFF044628B30221083007F08E
:101F5000A5F9012D024615D10B20FFF771FF507036
:101F600015702146002242F20C00FFF7A7FF04463D
:101F700030B9012D09D14FF480710848FFF719FFDE
:101F8000204638BD00234370EAE76FF480710348B0
:101F9000FFF71EFFF4E76FF03604F1E7E8290020B1
:101FA00070B5154D062205F108010646FFF7A3FEA0
:101FB0000446D8B1062142F20500FFF74FFF044660
:101FC000B0B106223146083007F06EF921460022F2
:101FD00042F20500FFF772FF044638B90622314687
:101FE00005F10800FFF797FE0123EB71204670BD55
:101FF0006FF03604FAE700BF7829002008B5092001
:10200000FFF71EFF024640B90820FFF719FF20B175
:102010001046BDE80840FFF78FBF002008BD012330
:1020200010B50621044600F8013B01F043FB18B946
:10203000A37963F03F03A37110BD000038B50C4DC8
:102040002B78012B10D1AB7903F0C003C02B0BD13F
:10205000681CFFF7A5FF044620B9042105F17000B4
:10206000FFF7A7FE204638BD6FF01504FAE700BF62
:1020700078290020F0B5BC4DD5F8B430996811F03E
:10208000010187B023D104AA40F60340FFF716FFF1
:10209000044600287CD1049B9B681B78A3B9B34AF3
:1020A00013602B46BFF35B8F53F8702FBFF35B8F2A
:1020B00002F00D02BFF35B8F53E8001F43E80020DE
:1020C0000028F9D1BFF35B8F049807F0B5F804AA94
:1020D000002141F20300FFF7F1FE0446002857D12A
:1020E000049BA348996808220131FFF714FE049865
:1020F00007F0A2F8214604AA41F20100FFF7DEFE34
:102100000446002844D1049883685A78AA73D97881
:102110009A7842EA01222A821A79EA73197ADA79DC
:1021200042EA01226A825A799B7942EA0323AB820E
:1021300007F082F80320FFF783FE014688B904AA5E
:1021400041F20900FFF7BAFE044608BB049B894828
:10215000996806220131FFF7DEFD04982C7007F024
:102160006BF804AA002141F20200FFF7A7FE044623
:1021700070B9049B8048996840220131FFF7CBFD7C
:10218000049807F059F8AB7E580604D46FF0120497
:10219000204607B0F0BD214604AA42F20300FFF733
:1021A0008DFE04460028F3D1049B744899680822E8
:1021B0000131FFF7B0FD049807F03EF8AB7E9906B9
:1021C00040F1908095F83A301A0700F1A780082175
:1021D00042F20100FFF742FE0446002800F0898029
:1021E0000821084407F05AF895F8403003F0060338
:1021F000062B14BF02234FF4C173002203701B0A85
:1022000043708270C270027142718271C271214644
:1022100042F20100FFF752FE04460028B8D108211F
:1022200040F60140FFF71AFE0646002861D008215B
:10223000084407F033F880234370022720230470FA
:102240008470047144718471C770C3712246314631
:1022500040F60140FFF732FE0446002898D10146BF
:1022600004AA4FF60140FFF729FE20BB049806F0B0
:10227000E3FF04AA21464FF60240FFF71FFED0B944
:10228000049B3F4899683A460131FFF744FD0498A2
:1022900006F0D2FF04AA21464FF60340FFF70EFED8
:1022A00048B9049B3748996801221144FFF733FD70
:1022B000049806F0C1FF0023072202A92A480293CE
:1022C000CDF80B30FFF717FD00283BD195F86030B3
:1022D000DB075BD42448FFF7A2FE044600287FF406
:1022E00057AF69E0022140F66D40FFF7B7FD0646A3
:1022F00010B96FF036044BE70221083006F0CEFF2C
:102300000123447003702246314640F66D40FFF7CA
:10231000D5FD044600283FF455AF39E704AA002153
:1023200042F21C00FFF7CAFD044600287FF430AFDC
:102330000498836853F8012F5B68C5E9202306F0F1
:102340007BFF44E7104B18689A8804909B79ADF89E
:10235000142004A9072204488DF81630FFF7CBFC9F
:102360000028B3D014E700BF7829002070000020B7
:102370008E2900207929002096290020F0290020AC
:10238000D7290020D6290020B8B1000001AA0021D9
:102390004FF60940FFF792FD00289BD10198816814
:1023A0004B786BB101230622023107482B70FFF7EF
:1023B000B2FC019806F040FFFFF740FE0446E7E656
:1023C00006F03AFF86E700BF7929002010B5FFF735
:1023D00051FE044630B902210648FFF7EAFC2046C8
:1023E000FFF70CFE044B1B681BB12046BDE81040F4
:1023F000184710BDE82900206C0000202DE9F04F9F
:10240000067D012E85B0044640F0988087683B78B1
:102410000E3B012B05D8404080F311884FF004009B
:1024200002DF00F1080318460221019306F045FF80
:102430003B783E2B61D1A7680198314606F03DFFFD
:102440003B78082B44D0092B67D0022B55D101983B
:102450003D4F06F03AFF804608F1FF385FFA88F8F2
:10246000B8F1FF0F49D0A6680198092106F025FFB1
:10247000337A3344711C93F809B07378023B012B13
:102480004FF0070202A856D8FFF745FC9DF8083028
:10249000023B8DF808303B68A3B1019806F01DFFA0
:1024A000337AB4F80CA0A3818146019B32783D6851
:1024B0004FFA8BF102A8A8472369A4F80CA013FADD
:1024C00089F3A360317A0198013106F0F6FEC3E783
:1024D000A6681E486FF02001FFF77AFC337843B9F5
:1024E000711C40221A48FFF716FC10211748FFF70D
:1024F00060FC184B1D68771C35B9204606F09CFE21
:10250000002005B0BDE8F08F32782B68002A0CBFA0
:102510003846002098476D68EEE70F4D2A68002A7C
:10252000EBD0A068037823B90130904700232B60DB
:10253000E3E70020F9E7FFF7EEFBACE706F07CFEEF
:102540006FF01500DDE700BF70000020E8290020D3
:10255000280000206800002024000020F8B5037D3A
:102560008668012B044605D0404080F311884FF067
:10257000040002DF8389012BF6D933780E3B012B4F
:10258000F2D800F108050221284606F096FE3378BD
:102590000E2B05D00F2B17D0204606F04DFEE3E79B
:1025A000A368032128461E7806F087FEA36821460B
:1025B0001878FFF71DFC16B10A4808F0CCF9204640
:1025C00006F03AFE0020F8BDA66804217778284678
:1025D00006F073FE21463078FFF70AFC002FEED09C
:1025E000EAE700BF002A0020084AD2F8B4303BB91D
:1025F000C16841B1016931B1C2F8B40018467047F1
:102600006FF0440070476FF0150070477829002084
:1026100038B50546054806F0F7FD044620B100210F
:10262000083006F0F7FD2575204638BDA42C0020A3
:1026300010B501464FF02003EFF3118083F31188AA
:102640000B4A0023D2F8A040C2F8A03080F31188D2
:1026500024B90120BDE81040FFF7DABF012204F1E0
:1026600008002275A381194606F0D4FD204610BD4E
:1026700078290020F7B51860C31D23F003030E4628
:102680001A80013A94B205460422002106FB040098
:10269000FFF76EFB4FF6FF77013CA4B2BC4201D1BD
:1026A00003B0F0BD04FB06602B180422801B0DEB69
:1026B000020128440193FFF72EFBEDE773B5046890
:1026C00006468CB1E31D23F00303042221460DEBE3
:1026D00002001D88FFF71FFB019B23B1DA1D22F0CA
:1026E0000302013D15803360204602B070BD70B515
:1026F0000C6806460D461CB1E31D23F003031C883D
:10270000042229463046FFF706FBF21D22F00302A1
:10271000631C13802E6070BD02FB01007047401ADD
:1027200080B2B0FBF2F0704710B5114401384FF69B
:10273000FF73013A92B29A4200D110BD11F8014DD7
:1027400000F8014FF5E710600860704710B5146895
:10275000206014686160106010BD884203D01AB117
:10276000436813607047002070470B68834207D0AE
:102770000AB1586810600BB11A680A6018467047B1
:102780000023FBE72DE9F047114FDFF848900426BE
:10279000013EF6B2FF2E19D033B24FEA830803EBA5
:1027A00043031D0104244FF00C0A0AE01AFB0451F4
:1027B0000A1D04EB08003A44394409EBC000FFF756
:1027C000C2FF013CE4B2FF2CF0D1E1E7BDE8F087A5
:1027D000F400002074000020F0B4124B05460F46B0
:1027E0000C26302472B1614306FB00142344597A4D
:1027F000187A814204BF0131197228463946F0BC6B
:1028000006F0DABB4C4306FB004423449C7ADA7A98
:10281000A24204D101329A72F0BC06F0FBBBF0BCBC
:10282000704700BFF4000020F8B505460E461C4670
:102830008AB1012362782078801A10F0030729D02A
:1028400003B3012F39D00132D2B22270314628466B
:1028500006F0E0FB1CE006F0CBFB0028E9D0314697
:10286000284606F0B7FB0028E3D030230C22734340
:1028700002FB0533124A1A44937AD27A9B1A18BF84
:102880000123D7E70232D2B22270D4E9020398477B
:102890000020F8BD002BF8D00132D2B22270042300
:1028A000302212FB06320C2313FB0523044A606816
:1028B0001A442146FFF74AFFC8E73846E9E700BF58
:1028C000F40000202DE9F04F00EB400389B01B011C
:1028D0004FF00008434E049305460424CDF80480CD
:1028E000013CE4B2FF2C0BD1019B002B72D0B8F15C
:1028F000000F6FD142462946284606F05DFB69E08D
:102900000DF1200B00230C274BF8043D4FF030094C
:1029100007FB04F309FB053031185A464968305863
:102920000293FFF71AFF049B17FB0437F319824643
:102930000393BAF1000F32D0079B1F785A78BF1A61
:1029400007F00307012F04D1013A5A70D3E90202BC
:102950009047079A13785278DBB29A1A02F0030272
:10296000012A05930DD0029B039909FB05303044E1
:1029700000224068FFF7F9FE079A059BC2F804A001
:102980005370029B09FB0533F1185A464968F05809
:10299000FFF7E3FE012F8246CBD1BCB9B0B930229C
:1029A0000C236A4303FB04223244917AD07A884292
:1029B00013D130226A4303FB042333441A7A597A31
:1029C00091421CBF5A724FF0010889E729462846F8
:1029D00006F020FB09B0BDE8F08FD1720122019210
:1029E000E7E700BFF400002010B5421E00200139C7
:1029F000C9B2FF2900D110BD12F8013F002BF6D05B
:102A00005C1E01302340C0B2F8E7F0B5427F046895
:102A1000064613460020FF2A01D10020F0BD02EB3C
:102A2000820504EBC5078A42D7F808C014F8355070
:102A3000604402D013462A46EDE7934200D17577F1
:102A40001BB203EB830304F833503B78FF2BE5D034
:102A500003EB830304EBC304A3686344A360DDE7D3
:102A600030B5551A15F4000F8368446909D125F073
:102A70007F421A44A2420ED9121B00248260446194
:102A800030BD8A1A22F07F42934201D99A1AF1E7A7
:102A90002244D41A0022A41A0022EFE7034600229F
:102AA0001A709A6A596208460AB1D96A1047704783
:102AB0002DE9F047857F01230446C3771DB9437F85
:102AC000FF2B02D1C577BDE8F08705F015FE6769D9
:102AD000667FD4F80080C71B27F07F47FF2E06D003
:102AE00006EB860608EBC6018B689F4218D2A27AD5
:102AF000E37A934205D10133DBB2022B08BF0023F6
:102B0000E372E37A04EB83030122DD60656A00234C
:102B1000E377AC46234604210320BDE8F047604735
:102B2000FF1A1D448A784B7818F836609B1ADBB27E
:102B3000012BD3D1D1F80C90013A8A70B9F1000F72
:102B4000CCD048696369CA8B281A184420F07F40AA
:102B50000B69496AC847C1E72DE9F04FC27F93B0BE
:102B60008346002A40F0A883436904930121837AB5
:102B70008177C07A984200F08C800B44DBB2022B44
:102B800008BF00238BF80A300BEB83030191D3F8C5
:102B90000C80049B434423F07F43CBF814309BF814
:102BA0001D300393DBF800300593DBF804300B9302
:102BB0009BF809300293002307934FF0FF0A029B12
:102BC000013BDBB2FF2B029366D19BF81D30039AC9
:102BD0009B1A18BF01230293019BCBB1DBF8009035
:102BE00000279BF81D50FF2D0BD02EB206EB86065A
:102BF00009EBC604A368434540F23281A3EB080306
:102C0000A360DDE901230399A94218BF134602938B
:102C1000DBF800300893DBF8043010939BF80930A0
:102C20000193019B013BDBB2FF2B019340F06881D4
:102C30009BF81D30039A9342079B40F032834BB9B7
:102C4000DBF804309BF809400193013CE4B2FF2C0F
:102C500040F09C8200238BF81E30029B4BB19BF806
:102C60001D30FF2B40F0E18205F02EFD08B9CBF8B6
:102C700018009BF81F30002B00F01E83DBF8244067
:102C80005B46012203210420A44613B0BDE8F04FA7
:102C900060470192904682E70B9B029A03EBC207C2
:102CA0007B680693F978BE788E4288D0069B387888
:102CB00006EB460212019D18731CDBB2984208BF56
:102CC0000023BB70069B9A5C032AECD9697801EB60
:102CD00081030A930A98059B03EBC004052A6378D5
:102CE000A078A3EB0003DBB20AD84BB1042A0CD1C5
:102CF0006A6852B9AA6842B9EA6832F07F4204D1E0
:102D000001212846FFF7CAFECCE7012B40F09D8049
:102D10005846FFF77AFE2B78A060042B064640F059
:102D20008680DBF81430089305F0E6FC089B0990D8
:102D3000C31A23F07F4343449E4202469EBF62690A
:102D4000921B9B18626896BF6361F31A0023002AE6
:102D500049D0A989002946D001F1FF3C1FFA8CFC1B
:102D6000A5F80CC09A42B4F81EE001D2F44502D393
:102D7000DFF8749231E0616A994E9A488E19864262
:102D800081BF01F1E87101F5D43101F5A5716162EE
:102D9000D4E908168CBF4FF001094FF00009761AEC
:102DA00091440EF1FF3E6662A3EB0903A4F81EE016
:102DB000D8E7D4E908160E4489498A487118814237
:102DC0008EBF002101214E4411440EF1010E8CBF33
:102DD000666266620B44A4F81EE0B4F81EE0F44597
:102DE000E7D8A4F81CC0AA881344A360EA886369E2
:102DF00013446361DDE908122046FFF731FEA26942
:102E00002B8913446A89A36193428CBF9B1A0023C8
:102E1000A361AB7B03B1E370059B0A9A03F832A070
:102E2000637895F801A001336370002169E7A37806
:102E300063706B789BF81C209A4201BFFF238BF8CC
:102E40001C300023CBF81830EFE704215B46DBF899
:102E5000244001220846A0470123BE700793AEE636
:102E6000DBF818209342A8EB03081F4429BFFF2377
:102E7000D31A8BF81C300023CBF81830A3691BB190
:102E80008BF81C50CBF818300022A26019F83630AD
:102E90008BF81D30D4F804C0BCF1000F2CD0A08BEF
:102EA000DFF840E1D4E908130B444D495918714546
:102EB0009FBFA3F1E873A3F5D433A3F5A5736362B1
:102EC00092BF019B63620023634410F1FF301A44F8
:102ED000E8D2049BA260DBF81410DA192046FFF751
:102EE000BFFDA38BE3830023E37009F836A063786A
:102EF00001336370AA4674E6A37863705546F9E718
:102F0000109B019A03EBC20304935B680A93049B32
:102F100093F80190BAF1FF0F40D00FFA8AF303EB58
:102F20008303089AD04612F833A002EBC3040025AD
:102F3000DBF800300B93FF232370A28BE38B9342CB
:102F400040F280809B1A9BB20C930FFA88F303EB3C
:102F50008303DB001193C8E009EB49030A9A1B01C4
:102F6000D51809F101025FFA82F9049A12784A45EC
:102F700008BF4FF000090A9AD35C032B0ED195F8D5
:102F80000180089B08EB880403EBC4046278A378F3
:102F90009A4208D001212846FFF780FD049B9B78C8
:102FA0004B45D9D13DE6EB68DBF8141063602B6923
:102FB0002362AB8AA383AB69A361EB69E3602B6AED
:102FC00023610026AB68A36066616A682046FFF74C
:102FD00047FD01236662E683E3704FF0FF0AA7E72F
:102FE0005A2B17FF592B177FB6562EFE6068002804
:102FF00000F0C780D4E90812B14B0A44B149D31894
:103000008B429CBFA2F1E872A2F5D432A3688BBFB9
:103010006262A2F5A57200226262034498BF012297
:103020001344E28BA3600132E283626993424FF062
:10303000000189BF9B1AD31AA36061619CBF6361C1
:10304000A16052E000237FE7B669091A46B9059FDF
:10305000B84200D23E1A0993059612F83E3053E06A
:103060000693F8E730B200EB800002EBC0070E9742
:10307000BF680F97774509D20E9FBF69002F54D1C3
:103080000F9EAEEB060E12F830604CE0FF264CE0CF
:10309000069B98456AD0069BFF2BA7D01E4633B2ED
:1030A00003EB83030593059A0B9B03EBC207FB8B92
:1030B000BA8B934288BF9B1A7A688CBF9BB200235D
:1030C000002A93D00C9A934290D8FA78E3789A42E7
:1030D0008CD231465846FFF798FCBB787B70059A36
:1030E0000B9BB86003F832A0B246119BDBF80020BE
:1030F000DBF81800059002EB030CFF209BF81D3055
:10310000DCF8081009930690FF2B06D003EB830E22
:1031100002EBCE06B068814296D8DCF818000D901C
:1031200001EB000E1E46FF2E9CD10D9828B105988C
:103130008142ADD3FF2E40F0BB800998CCF8081037
:10314000834218BFBDF924008CF8003016BF00EB95
:1031500080008BF81D8002F83080FF2B06D003EB37
:10316000830302EBC3039A68511A9960A378013371
:1031700063700021002D3FF4CDAE2846FFF78EFC92
:10318000C8E60121F6E70123029359E5019B03EB11
:10319000C4056E686B78EA789A423FF456AD03EB4B
:1031A00043031A01B318B25C012A24D0022A29D1A0
:1031B000D3E9019099F80020D3F80CE0DBF800C0C7
:1031C000DBF81410FF2A02D00768B94223D09BF81D
:1031D0001D2001600021FF2A09D002EB82080CEBC0
:1031E000C80ADAF808000144DAF81800D0B189F802
:1031F0000020CEF8001000225A629A6A12B1D96AF1
:10320000002090476B782A780133DBB29A4208BFDE
:1032100000236B70BEE702EB8202DEF800101CF8A0
:103220003220D8E71CF83820D5E7039BFF2B07D1C5
:1032300005F062FA044605F039FA08B9CBF81440F3
:103240009BF81D30DBF8002003EB830302EBC30384
:103250000A269D6805F050FADBF81440031B23F0A2
:103260007F430333AB422CBFE418641924F07F443E
:103270000746DBF828302046984705F03DFAC01B8A
:1032800020F07F40E41B033024F07F44A0427FF60F
:10329000F0AC013EDED1404080F311884FF00400D5
:1032A00002DF002B3FF46FAF00238BF81E30D6E413
:1032B000B0457FF4F4AE59E713B0BDE8F08F00BF1E
:1032C0005A2B17FF592B177FF0B51C4E059F9DF801
:1032D0001840DDF81CC02C25454306EB050E725145
:1032E0008EF808108EF80930CEF80470013BDBB27E
:1032F000FF2B13D104BB2C2358433318089A1A62AE
:10330000099A5A6218300A9A9A6232184FF6FF7177
:103310003450918020465C615C81F0BD1AB207EBAD
:10332000C201C1F804C017F8322002EB4201A41A0E
:103330000CEB011CE4B2D9E70120EEE7B401002058
:10334000044A2C2303FB0020007A003018BF012020
:10335000704700BFB4010020074A2C2100FB012365
:1033600010B45C6A2CB1A44601220321022010BCD7
:10337000604710BC704700BFB40100202DE9F04148
:10338000224C2C2700FB07480DB2D8F8040000EBB4
:10339000C50C10F835009CF80340661CF6B2B0422C
:1033A00098BF00269CF80100B0422DD0DCF8040044
:1033B00004EB4404250144194FF0030E00F805E026
:1033C0006360069BA360079BE360089B23610A9BE5
:1033D000A361BDF82430A3820B9BE3610C9B2362A5
:1033E000022363620D9BA3620E9B6270E3628CF802
:1033F0000360D8E90835084698474346002204216F
:10340000A847606ABDE8F0810120FBE7B401002015
:103410002DE9F843224C2C2700FB07490DB2D9F8BF
:10342000040000EBC50C10F835009CF80340661C46
:10343000F6B2B04298BF00269CF80100B0422DD0F1
:10344000DCF8040004EB4404250144194FF004089F
:1034500000F80580A380BDF82030E380BDF824305B
:103460002381BDF828306381BDF82C30A3819DF8FD
:103470003030A373022363620D9BA3620E9B6270C4
:10348000E3628CF80360D9E90835084698474B4653
:1034900000224146A847606ABDE8F8830120FBE7A7
:1034A000B40100202DE9F0411A4C2C2600FB0648FF
:1034B0000FB2D8F8040000EBC70C10F837009CF8E6
:1034C0000340651CEDB2A84298BF00259CF801009E
:1034D000A8421CD0DCF8040004EB440424010719C2
:1034E0004FF0050E00F804E07A700222C7E90923C4
:1034F000069BFB628CF80350D8E9083408469847CD
:10350000434600220421A047786ABDE8F0810120EB
:10351000FBE700BFB40100202DE9F0411C4C2C2733
:1035200000FB07480DB2D8F8040000EBC50C10F8FA
:1035300035009CF80340661CF6B2B04298BF0026E6
:103540009CF80100B04221D0DCF804E004EB440414
:1035500025010EEB050402200EF80500C4E9012345
:10356000069BE360079BA362FF25089B6570606272
:10357000E3628CF80360D8E908350846984743466B
:1035800000220421A847606ABDE8F0810120FBE722
:10359000B40100202DE9F0411A4C2C2600FB06480E
:1035A0000FB2D8F8040000EBC70C10F837009CF8F5
:1035B0000340651CEDB2A84298BF00259CF80100AD
:1035C000A8421CD0DCF8040004EB440424010719D1
:1035D0004FF0010E00F804E0FF2078700220C7E9E8
:1035E0000902FB628CF80350D8E908340846984772
:1035F000434600220421A047786ABDE8F0810120FB
:10360000FBE700BFB40100202DE9F041084C2C2558
:1036100005FB0043D3E9083706460846984706FBF2
:103620000543BC4600220421BDE8F041604700BFCD
:10363000B401002005F060B8401A20F07F407047C8
:1036400008B50346012B08460ED833B119B106223E
:103650000649FEF760FB054807E019B10622044958
:10366000FEF759FB024800E0002008BD12020020CE
:103670000C02002070B506460D4604F0ABF9044676
:1036800010B10C24204670BD04F0B8F910F0060FFC
:10369000F7D1062229461EB10248FEF73CFBF1E7AE
:1036A0000148FAE7120200200C02002000230370F8
:1036B0000B70704773B50C464618351B8CB1FDF77F
:1036C00019FD032C019007D904220DEB02012846B5
:1036D000FEF721FB043CF0E7224601A92846FEF74D
:1036E0001AFB002002B070BD08B50248FEF77CFF4F
:1036F000002008BDCCB60000838910B504469BB1FC
:10370000037D8BB900F082F930B183681B780E3BE2
:10371000012B06D8FEF722FF204605F08DFD002084
:1037200010BDFEF76BFEF7E76FF01500F8E700003D
:1037300073B51C4D00264FF0FF31284606F03EFEC3
:10374000044618B300F032FD0228019421D8012864
:103750000EBF00214FF0FF310120FEF759FF044654
:1037600018B10146019800F039FC019B0021D8886E
:1037700004F00AFA02A850F8043D1E6004F0A4F90F
:1037800024B1A389204653B1FEF738FE07F078F83C
:10379000D1E7404080F311884FF0040002DF05F0CC
:1037A0004BFDF3E7742C002037B50C4C0C4D0DF19C
:1037B000020101A804F050F90028F8D1019B33B1AF
:1037C00004F096FB0199284606F0D4FDEFE74FF090
:1037D000FF31204607F0E6F8E9E700BF5C2C002047
:1037E000742C002010B5144886B004F025FC044663
:1037F000F8B900F0FBFC6FF00903CDE902434FF488
:10380000E0720E4B0E490F48CDE90444CDE9004467
:1038100007F08AFA6FF00703CDE90243CDE90444CB
:10382000CDE90044084B094909484FF4806207F08C
:103830007BFA204606B010BD5C2C0020A9370000A2
:1038400048120020200F002031370000081400200B
:10385000B00E0020C0F307230870000C8870000A27
:103860004B70C870704738B508300D4602211446B9
:1038700005F014FD0570447038BD000038B50446ED
:103880004FF0FF300D46FEF7D3FEEA1C2060D2B2A7
:103890000E21FFF7E8FF20680321083005F0FEFC49
:1038A00001230370054B1B88A0F8013020682946CE
:1038B0000830BDE8384005F0F1BC00BF1802002018
:1038C00070B50446154601320E460834D2B23E2188
:1038D000FFF7C9FF0121204605F0E0FC06702946EC
:1038E0002046BDE8704005F0D9BC00002DE97848BD
:1038F00004461846154B1646D3E900234FF0000B3B
:1039000003F0005C5BEA0C030D461DD0104BD3E9BD
:1039100000234FF0000C02F0080B5BEA0C0313D0FD
:103920000B220421FFF7CCFF08220470A0F80160ED
:10393000033024B9291DBDE87848FEF7ECB9002111
:10394000BDE87848FEF714BABDE87888302A002030
:10395000382A002070B503788AB004460E4607ADB9
:10396000032B20D8DFE803F002191B1D114928465C
:10397000FEF7AAF962780492A2780392E2780292A2
:103980002279019262790092A37905950A4A1B2156
:103990003046FDF7AFFA0AB070BD0849E7E70849BD
:1039A000E5E70849E3E7084A0A212846FDF7A2FAB5
:1039B000E0E700BFEBB6000014B70000F2B600006D
:1039C000F9B6000003B700000DB7000010B583780A
:1039D0009A068AB013D0C378DB0710D501460AAC2B
:1039E00011F8043BC3F3801304F8243D06220DF1C3
:1039F0000500FEF790F903A92046FFF7ABFF0AB0D8
:103A000010BD03460068596870470000F0B5818911
:103A100099B00025022904460D9502D8002019B05E
:103A2000F0BD8368C54E1A7858789B7842EA002228
:103A30008B423280F2D8032104F1080005F03DFCEE
:103A40003388C3F309029B0A042B63D007D8032BE6
:103A500024D001210DA8FFF711FF0123CCE1082B91
:103A600000F0D9803F2BF4D1013A092AF1D801A303
:103A700053F822F0FD3D00002B3E0000533E0000B5
:103A8000533A0000533A0000973E0000533A0000BA
:103A9000693E0000A13E00000D3F0000032A14D043
:103AA00008D8012AD5D1A068FFF7ABFFA44BC3E922
:103AB000000103E02D2A17D0632ACAD101210DA8E5
:103AC000FFF7DCFE05700D98A9E79D4B4FF0FF3026
:103AD00041F6FF71C3E900019A4B1F200021C3E9A1
:103AE000000103F01DFFE9E7A36804210DA81D886C
:103AF0009F78FFF7C3FEAEB20446C21C394630467B
:103B000003F0A0FF002814BF022300232370A4F8B1
:103B10000150D8E7013A082A9BD801A353F822F0B4
:103B2000453B00006F3B0000E33B0000533A0000C0
:103B3000533A0000533A0000533A0000533A000051
:103B4000FF3B000009210DA8FFF798FE002303703A
:103B50008370C3706FF00E034371052309228371D4
:103B60004FF0FF3342700271C3710372ABE7412122
:103B70000DA8FFF783FE00210446402200F8011B38
:103B8000FEF7F6F8E378217FA27E63F07F03E3700F
:103B9000A37963F03F03A371E37A43F00403E37274
:103BA000E37B43F02803E373237C43F00203237495
:103BB000E37D43F00403E375E37E61F03C0163F0D1
:103BC0003C032177E376617F94F8273041F00801C8
:103BD00062F0080263F07F036177A27684F82730F1
:103BE00071E709210DA8FFF749FE002104460822CC
:103BF00000F8011BFEF7BCF86023637163E707213F
:103C00000DA8FFF73BFE0146002301F8013B1846D3
:103C1000FFF716FD57E70A2A00F0E18027D8052AAA
:103C200000F0818012D8022A5FD0032A69D0012ACD
:103C30007FF40FAFA068FFF7E4FE424BC3E9000139
:103C400001210DA8FFF71AFE0023D5E0072A00F096
:103C50005581C0F0A680082A00F0BB80092A7FF4B5
:103C6000F8AEA368591C187804F0BEFBE8E7122AE6
:103C700077D010D8102A67D06FD80F2A7FF4E9AE1A
:103C800002210DA8FFF7FAFD00230370044604F09B
:103C90005DFC607017E7182A67D015D8172A7FF4E3
:103CA000D8AEA06800230EAA00F1100104F05EFD5A
:103CB00011210DA8FFF7E2FD002300F8013B1022BF
:103CC0000EA9FEF728F8FEE61C2A59D04B2A7FF4ED
:103CD000C0AE03210DA8FFF7D1FD0146002301F876
:103CE000023B0130FFF7E2FCEDE604210DA8FFF7EF
:103CF000C5FD002303701B22837002234270C37032
:103D0000E1E609210DA8FFF7B9FD002104460822CC
:103D100000F8011BFEF72CF80C2363704023A370FE
:103D20000123E370CFE6A1680120FFF7A3FC04465E
:103D300001210DA8FFF7A2FD0470C4E618020020BF
:103D4000302A0020382A002001210DA8FFF796FD17
:103D5000044604F0FDFB2070B5E6A06804F00EFCFC
:103D6000E5E7A06804F042FCE1E709210DA8FFF7B0
:103D700085FD002300F8013B0821FFF79BFCA2E62C
:103D800009210DA8FFF77AFD01460022044601F83B
:103D9000012B0320FFF75EFD611D1046FFF75AFD62
:103DA00091E6A068002103790288CDE90911CDE9E7
:103DB0000711CDE90511847B0494447B0394C41D51
:103DC00002948479019440790090084604F0C2F985
:103DD000ADE7A368591C187804F0AEFA30E7A36881
:103DE000187804F047FB012104460DA8FFF746FDB3
:103DF000002C14BF0C230023037064E60D210DA8D2
:103E0000FFF73CFD02224270C270012282710C2237
:103E10000023C271632203708370037143710372C4
:103E200042728372C37203734DE641210DA8FFF7FE
:103E300025FD00210446402200F8011BFDF798FFF4
:103E4000637863F058036370A37843F00303A370AF
:103E500039E609210DA8FFF711FD002100F8011B2B
:103E60000822FDF785FF2EE65B4B0EAA03F128061C
:103E7000154618685968144603C40833B3422246ED
:103E8000F7D129210DA8FFF7F9FC002300F8013B29
:103E90002822294615E7A1680020FFF7EBFBCFE6B3
:103EA0004FF08053D3F8A420013206D1D3F8A830C4
:103EB0004FF6FF729BB2934220D04FF08055D5F859
:103EC000A030DB071AD518210DA8FFF7D7FC002674
:103ED0000123044643700670D5F8A400A11CFFF727
:103EE000B9FCD5F8A830A371C3F3072363F03F03EF
:103EF000E3711022314604F10800B2E702210DA857
:103F0000FFF7BCFC002303704370DCE521210DA802
:103F1000FFF7B4FC0346002203F8012B4FF0805258
:103F20000446D2F8901001314BD0D2F894100131F0
:103F300047D0D2F89810013143D0D2F89C1001310B
:103F40003FD0D2F890001946FFF784FC611DD2F8EB
:103F50009400FFF77FFC04F10901D2F89800FFF705
:103F600079FC04F10D01D2F89C00FFF773FC4FF0CF
:103F7000805204F11103D2F88010013127D0D2F819
:103F80008410013123D0D2F8881001311FD0D2F82B
:103F90008C1001311BD0D2F880001946FFF75AFC73
:103FA00004F11501D2F88400FFF754FC04F1190163
:103FB000D2F88800FFF74EFC04F11D01D2F88C0006
:103FC000ECE6102200211846FDF7D2FECFE71022C2
:103FD0000021184645E700BF37B700002DE9F04142
:103FE0000379012B8AB004460D4600F1080800F061
:103FF0009B80023B032B00F2CD80DFE803F00253ED
:10400000535F674B03934FF60473ADF810300223F0
:104010008DF81230634BD3E90023002003F00051E8
:1040200050EA01033BD0604BD3E90023002102F0AA
:10403000020050EA010332D0227A637A02F00F02C2
:10404000012A1ABF9E1FF6B20026234406F10B0276
:10405000D2B2022128469F7AFFF732FC0123037077
:10406000237A0AAA03F00F031344054613F81C3CF5
:104070004370237AC3F380138370062204F10A018C
:104080000330FDF748FE0A3505F8016C7F427FB228
:10409000324608F108012846FDF73DFEAF550AB04B
:1040A000BDE8F081037A03F00F03072BF7D1437AC1
:1040B000002BF4D04046FFF789FCF0E7394BD3E9F9
:1040C000002300F10A0603F00051002050EA01032A
:1040D00008D0354BD3E90023002102F4802050EAB8
:1040E000010310D1237A0AACC3F3801304F8243DF2
:1040F000314606220DF10500FDF70DFE03A920460D
:10410000FFF728FCCBE7082213212846FFF7D8FB4E
:1041100000230370237AC3F38013437006223146D1
:104120000230FDF7F8FDBAE7C17AC68809290BD03D
:104130000C2910D007292DD1037B0E2BAFD12B4694
:10414000324600211A2003E02B4632464146002029
:10415000FFF7CCFBA3E7134BD3E900234FF0000894
:1041600002F4006757EA080399D008222846FFF7AF
:104170007AFB0821681805F091F800230370A0F875
:104180000160237BC370B4F80D308380B4F80F3026
:10419000C38084E7404080F311884FF0040002DFC1
:1041A000000103FF302A0020382A00200379012B68
:1041B0000FD00A2B15D8012000FA03F313F4B06FC7
:1041C00012D113F03C0F10D183F0400343F3801061
:1041D0007047037A03F00303032B0CBF0220032074
:1041E00070474FF0FF30704702207047064B4FF08A
:1041F000FF3041F6FF71C3E90001044B1F2000218D
:10420000C3E90001704700BF302A0020382A00208F
:1042100020BF40BF20BF7047F0B50D4B89B00546A9
:104220000E4601AA03F1180718685968144603C41A
:104230000833BB422246F7D11B88238008AB1D44BC
:1042400015F81C0C831B5842584109B0F0BD00BF43
:10425000BFB100000860704718B90B6843F0004315
:104260000B60704718B90B6823F000430B60704770
:1042700070B5031D451E00249D4201D1204670BD2E
:1042800015F8016F0022A018082AC0B201D1044617
:10429000F2E716F0010F03D00029F0D00139C9B2BE
:1042A00076080132EFE7000010B50C4A92F83A3177
:1042B00092F839118B4238BF92F8384192F839118F
:1042C00038BF1B195B1ADBB298429BBF92F83911B9
:1042D000D2F83431002053F8210010BD1C02002018
:1042E00030B590F85C3090F85D10994228D190F983
:1042F0001D30002B26DBC48C828CA0F86440C48D5A
:10430000A0F8622054437D2262434FF47A7492FBFA
:10431000F4F2A0F8662090F86020012565F3010210
:10432000D2B2002342F00402013980F87050C36613
:1043300080F8602080F85E5080F85D10184630BD2F
:104340000120FCE70220FAE72DE9F84F0C789442AF
:1043500081460F4690463DD01F4ED6F8683133F85F
:104360003430038000254FF0020B06F5AE7A22B2FE
:10437000D6F86801B9F800C000EBC20130F832206D
:10438000944520D14868012820F003030AD9F3B1ED
:10439000021D1CD04279D2B1027902F00302013A27
:1043A000012A14D8012215444A60EDB213B15146D6
:1043B000FEF79DF9013496F86C21E4B2A24208BFE1
:1043C00000244445D3D13C702846BDE8F88FC1F89D
:1043D00004B0EBE70025F7E71C02002010B5094BFD
:1043E00093F81021824204460AD902464FF48271A2
:1043F000D3F80801FEF790F910B1038CA34200D066
:10440000002010BD1C0200202DE9F04186B00223DF
:10441000052805460F4602930ED0062800F08D8031
:1044200040F28580073880B2FFF7D8FF002800F0FF
:10443000D680D0E900680FE06A4BD3E9066802AB8A
:1044400000930A46684B03210020FFF72BF802284F
:1044500066D0029B002B67D1624CA37C03F0FF0067
:10446000002B64D106AB0222A57443F8102D032162
:1044700000932A465C4BFFF715F8022861D0029B97
:10448000002B45D1237CAB4202D0637CAB423BD1B5
:1044900006AB022243F80C2D002200930321524B5D
:1044A0001046FEF7FFFF022807D101221146032024
:1044B000FEF792F9039B022B39D0039800285CD1B8
:1044C00002230493237C002B31D004AB0093012200
:1044D000454B20740321FEF7E5FF022807D1012296
:1044E00011460320FEF778F9049B022B1FD0049A93
:1044F000002A34D126F00046B0453CD93B4B11464A
:104500000320FEF791F990B9A37C0BB90123029324
:104510000023A374029806B0BDE8F081FFF778FE8F
:10452000029B022BFAD094E7029B012B94D04040CF
:1045300080F311884FF0040002DF2A4BD3E934687E
:104540008AE7637CAB4204D1012211460320FEF7C7
:1045500043F9029B022B92D1FFF75AFEF9E7049B25
:10456000012BE4D100221146204B0320FEF75CF919
:1045700002460028DBD11E4BC1E7039D012DD6D199
:10458000FF2F19D006AB022243F8042D032100931C
:104590003A46154B0020FEF785FF022807D12A4630
:1045A00029460320FEF718F9059B022BBFD0059B77
:1045B00013B1059B012BBAD1E37C002BA4D00D4B8A
:1045C00004229A60002211460320FEF72DF90028EC
:1045D000ADD1E37C002B97D0FFF71AFEF9E701205D
:1045E00099E700BF1C02002055420000802A0020ED
:1045F000202B0020B02A00202DE9F04F8BB00024A2
:10460000FF25DFF814918DF81F50804693461F4612
:1046100001F1040A1C60089426460223099309ABA1
:1046200002933B4B019308AB00930DF11F025B46D5
:1046300041460020FEF770FF02280BD0099B6BB1AA
:10464000404080F311884FF0040002DF4146002013
:10465000FEF7DAFF099B022BF8D0EFE79DF81F2049
:10466000FF2A4DD0062AD8D999F8103107339A423B
:10467000D3DA073A92B24FF48271D9F80801FEF703
:104680004BF80028C9D090F91D30002BC5DBD0E9CC
:10469000003C002B089A12DA816823F000438C4515
:1046A0002CBF62445218D21AC168FF2D01F10401D7
:1046B0000B4408D19DF81F501C461646ADE76345D4
:1046C00038BF6346F0E73146104605930492FEF783
:1046D000B3FF04EB0A018842DDE90423EAD90D485F
:1046E0003444A4FB0001072303FB041106A3D3E910
:1046F0000023FBF7C5FD803038600BB0BDE8F08FBC
:10470000FF2DECD1F9E700BF00CA9A3B0000000082
:10471000554200008D49FD1A1C02002070B5047836
:104720000A78C4F38013B3EBD21F19D104F00F043D
:10473000012C00F1020501F1080608D006223146DD
:104740002846FDF7D8FAB0FA80F0400970BD06227D
:1047500031462846FDF7CFFA0028EFD12046F5E78D
:104760000020F3E70B4A92F8783192F879119942D8
:104770000ED192F8783102EB4303A3F8720192F85C
:1047800078310133DBB2032B08BF002382F8783184
:10479000704700BF1C020020404080F311884FF09A
:1047A000040002DF08B508B1FFF7F6FF08BD0000FE
:1047B000012808B5094B07D19A7C052A02D10022AD
:1047C0009A7408BDFFF7E8FF1B7C052BF9D1404028
:1047D00080F311884FF0040002DF00BF1C020020AC
:1047E000012808B5094B07D19A7C062A02D100227C
:1047F0009A7408BDFFF7D0FF1B7C062BF9D140400F
:1048000080F311884FF0040002DF00BF1C0200207B
:1048100008B528B1034B9B7C052B01D0FFF7BCFFEB
:1048200008BD00BF1C02002008B530B1034B9B7CC3
:10483000C9B2994201D0FFF7AFFF08BD1C020020AA
:10484000044B1B7D23B1012100220846FDF7C4BFA4
:10485000704700BF1C020020062810B50C460AD97C
:10486000094BC21F92B24FF48271D3F80801FDF7D1
:1048700053FF206010BD052804D00628034818BF48
:104880000020F7E70248F5E71C020020EC020020B8
:104890003402002008B50A4B00221A70094BA3F11C
:1048A0001001012818BF0B461146FDF7BDFF28B1C6
:1048B000404080F311884FF0040002DF08BD00BFC4
:1048C00024040020002B0020002208B51146044BD0
:1048D0001046FDF7A9FF08B1FFF75EFF08BD00BF56
:1048E000502A0020002208B51146044B1046FDF75F
:1048F0009BFF08B1FFF750FF08BD00BFD02A002082
:1049000008B50A4A137838B1591C117063B90120EF
:10491000BDE8084003F088BB0BB9FFF73DFF013B42
:10492000DBB21370002BF3D008BD00BFD003002012
:104930000020FFF7E5BF0000C0B208B5031F012B40
:1049400001D9FFF729FF084A137D13B1043B012B5E
:1049500006D804F0CDF828B9BDE8084004F096B8B0
:104960001075F9E708BD00BF1C02002038B50546E8
:104970000C460021084603F0EFFF95F8A830DB064F
:104980004FF001020DD51F21082004F02BF822461C
:10499000002105F1A90004F05FFABDE8384004F0F9
:1049A0004FB808201B2104F01DF82046F5E7000051
:1049B00038B5104A92F8703192F86C410133DBB28D
:1049C0009C4208BF002392F86F419C4201D1FFF73F
:1049D000E3FE92F87051D2F8684124F8350092F85D
:1049E000700104EBC004616082F87031BDE83840AA
:1049F00003F01CBB1C0200202DE9F047254D0646A4
:104A0000A846002795F86D3195F86E219A4236D068
:104A100095F86D91D5F864A1D5F808013AF83920D8
:104A20000AEBC9034FF482715C682760FDF774FEDE
:104A300003463AF839001A8C824222D1D3F8F82082
:104A400042B9D3F8EC20C3F8F8401AB9C3F8EC40E7
:104A5000C3F8FC20D3F8FC2002B11460C3F8FC407A
:104A600098F86D3198F86C210133DBB2013E9A421F
:104A700008BF002316F0FF0688F86D31C2D1BDE8EB
:104A8000F087237967F3010323712146FFF790FF35
:104A9000E6E700BF1C02002073B501220446114660
:104AA0000020FDF799FE94F82020002142F2EA232D
:104AB000073200930846374BD2B2FEF7F3FC30F0D2
:104AC000020105D0404080F311884FF0040002DF5E
:104AD000314B1A7D052A1D461BD1228C187C0732CA
:104AE000904216D1197442F2FB2300930122294B04
:104AF0000846FEF7D7FC30F00202E3D142F202335F
:104B000000931146234B1046FEF7CCFC30F0020315
:104B1000D8D1D4E93B13994203D0D4F8F830994264
:104B200001D11E4E10E00B796FF301030B710B687E
:104B3000C4F8EC30208CFFF73BFFEAE7036831460E
:104B4000C4E93B33FDF7D3FDD4F8EC0018B1D4F839
:104B5000F8309842F2D10023C4E93C33D4F8EC1089
:104B600051B94FF6FF732384D5F88031A34208BFB3
:104B7000C5F8801102B070BD0B796FF301030B71A2
:104B80000B68C4F8EC30C4F8F830208CFFF710FF45
:104B9000E4E700BFA54700001C02002070030020CE
:104BA00038B505460C460021084603F0D5FE95F8B9
:104BB000A8309B064FF001020CD51F21082003F0FE
:104BC00011FF214605F1CA0004F082F9BDE8384022
:104BD00003F03CBF08201B2103F004FF2046F5E74B
:104BE000262810B504460BD027280BD025280BD13A
:104BF000022003F0C7FE2046BDE8104003F0C8BE07
:104C00001A20F6E75020F4E70A2802D802304000C4
:104C1000EFE7272801D80330F9E7FFF7BDFD0000D3
:104C200038B52A4C94F8783094F879209A4206D016
:104C30000133DBB2022B08BF002384F8783094F8EC
:104C4000C83094F8C9209A4206D00133DBB2022B57
:104C500008BF002384F8C83094F878202A23272539
:104C600015FB0235601903F0F1FE635D03F00F03DD
:104C7000022B23D0072B21D002239620237503F08B
:104C8000EFFF002003F05CFF94F82830C3F302022A
:104C9000D3B21946002011F0010F00F1010512D026
:104CA000013B134094F82820C0B263F3020284F859
:104CB00028202530BDE83840FFF792BF0323237535
:104CC00003F054FFE0E749082846E4E71C0200200F
:104CD00073B5164602AA1C46054642F8046D2731F4
:104CE0000120FFF789FC2368FBB10198831B1B029D
:104CF00001D5FFF751FD3146FEF79EFC02461048F4
:104D00000723A2FB000103FB02110BA3D3E900233D
:104D1000FBF7B6FA236818440028206005DB40F250
:104D2000E24068432368834201D802B070BD1B1A79
:104D30002360F7E7AFF3008000CA9A3B0000000051
:104D40008D49FD1A13B500F16C030446826FC168EA
:104D5000808CFFF7BDFF02A9E36E606F40F2E24274
:104D6000B3FBF2F3022221F8023DFCF7D4FF02B0BC
:104D700010BD00001FB53E4C20B1A37C052B75D0A3
:104D8000FFF70AFD237C052B02D0637C052B65D140
:104D900004AB022243F8082D002200930121354B79
:104DA0001046FEF77FFB02280DD00298C0B1029892
:104DB000012819D1E37C002B50D02F4B04229A609C
:104DC0000022114646E0012211461046FDF704FD7F
:104DD000029B022BE9D101210020FEF715FCF7E729
:104DE00002230393237C2BB9404080F311884FF0BA
:104DF000040002DF03AB01222074114600931D4B17
:104E0000FEF750FB02280FD0039AD2B1039C012C6D
:104E1000EAD100221146194B2046FDF705FD024656
:104E20000028E1D1164B13E0012211461046FDF790
:104E3000D3FC039B022BE7D101210020FEF7E4FB0A
:104E4000F7E7A369E16923F000438B42EAD20B4BF9
:104E500011460120FDF7E8FC0028C5D10022094BCE
:104E600011460120FDF7E0FC0028BDD104B010BDC3
:104E70001C02002055420000A02A0020702A0020B9
:104E8000102B0020402A002070B5164C037894F8AF
:104E9000E120DB09B3EBD21F05460E4607D094F89C
:104EA000E100C0F3011010F002000BD170BD00F161
:104EB0000801062204F1E200FCF71DFF0028EED1F4
:104EC0000120F3E795F90030002B09DA6B7B03F042
:104ED000C003402B04D1002EF2D001203070E5E752
:104EE0000020E3E71C02002010B5164A92F8393181
:104EF00092F83A11994201D1FFF74EFC92F839111C
:104F0000D2F8343153F8211092F8703108680B70E0
:104F100092F8393192F838410133DBB29C4208BF34
:104F2000002382F8393102F5A472FDF70FFC28B98D
:104F3000404080F311884FF0040002DFBDE81040CC
:104F400003F074B81C02002010B50120FFF7ACF983
:104F5000044608B9FFF720FC4FF6FF73C380062311
:104F60000371102200210B30FCF702FF3C23E37297
:104F7000BDE81040FFF7B8BF03460A4600F19C01A8
:104F8000D0F89C0010B508B9FFF706FC1C8CA3F8FC
:104F9000A24083F8A42007240A4A83F8A04092F88C
:104FA000704183F89C4002F5A472FDF7CFFB28B94D
:104FB000404080F311884FF0040002DFBDE810404C
:104FC00003F034B81C020020404080F311884FF0F9
:104FD000040002DF70B506460320FFF765F90446BA
:104FE00020B34FF6FF73C380114B93F8E1305A079B
:104FF00018D0C3F30203DAB2012A03D0042A02D084
:10500000FFF7E2FF0323237104F1080566B103F003
:10501000C5FD00F07F00637A1D44A870FFF764FFB0
:10502000002070BD0223EEE77F20F4E70120F8E7BF
:105030001C02002030B50468002C89B019DAD0E9D0
:10504000013524F000449D4234BFE41A641B0A4B2E
:105050000593A4B200230690CDE90333CDE90143C3
:1050600018460094FEF7D4F930F0020301D0FFF7A0
:1050700093FB09B030BD00BF6542000037B502ADFB
:10508000104B45F8043D044603F04CFC002003F0AF
:1050900073FC0D4803F010FC0121204603F05CFC7A
:1050A000284603F087FC620002F0FE02252108205A
:1050B00003F098FC054940F25B6003F023FD03B068
:1050C00030BD00BFD6BE898EE95F00005555550042
:1050D00008B5054B0022986011461046FDF7A4FB69
:1050E00008B1FFF759FB08BD902A00202DE9F04FC9
:1050F00014681D688DB0002C81460B9190469B462C
:105100009DF85CA003DA169CAC4238BF2C46AC423A
:105110004E4F1BD941F27453CDE907734C4B00211C
:10512000CDE90413631B009306914B46CDE90211B0
:10513000019101220846FEF721F930F002032BD03D
:10514000404080F311884FF0040002DF1DD200239D
:105150001A4619461846FFF7B7FB41F28953CDE9C5
:1051600007733C4B00212C1BCDE9041306914B46E1
:10517000CDE90211CDE9004101220846FEF7FEF813
:1051800030F00203DCD12C460BE000231A4619460E
:105190001846FFF799FB00231A4619461846FFF7F1
:1051A000A1FB2D4E0B9BF36041F2A153CDE9077398
:1051B000199B06930022189B0593CDE903224B46C9
:1051C000CDE90122009411461046FEF7D7F830F0E1
:1051D0000203B5D10520FFF77BFFD6F87C31AB4247
:1051E00023D0CBF80030D8F80030002BBCBF23F020
:1051F0000043C8F80030D8F80020D6F87C118A4265
:1052000038BF0A4641F2CF51A3B292B2CDE905713F
:105210000021CDE901230092CDE903115246084651
:10522000FEF7F6F830F002038AD1FF20FFF7E4FB27
:105230000A4B012211460020C3F808A0FDF7F4FA3A
:1052400000287FF47DAF0DB0BDE8F08FA5470000CA
:10525000C9480000E54800001C020020302B002057
:105260001FB50B4A137C03F0FF040BB1FFF794FA50
:10527000052313740394074CCDE90134136A00939A
:1052800002F11C031832FFF731FF04B010BD00BF5C
:105290001C0200201555000007B50520FFF718FF78
:1052A00041F69303002100930522064B0846FEF7C2
:1052B000F9F830F0020301D0FFF76EFA03B05DF8A1
:1052C00004FB00BF754D00002DE9F843214D95F812
:1052D0003A4195F8383195F84C910134E4B2A34243
:1052E00008BF002405F5A07705F59478B9F1000F03
:1052F00003D095F839319C4201D1BDE8F883384696
:10530000FDF7DCF906460028F7D04046FDF7D6F950
:1053100028B930461049BDE8F843FDF7E8B9066002
:1053200095F83A21D5F8343143F8220085F83A410E
:1053300095F838310134E4B2A34208BF002495F84F
:105340004C3109F1FF39013B85F84C315FFA89F99D
:10535000CCE700BF1C0200205C03002010B52C4CE1
:1053600094F81021002A37D004F586734FF4827127
:10537000D4F80801FDF77EF9264B94F83221B4F8F1
:105380003011D4F82401FDF775F994F8381194F828
:105390001021214BD4F83C010A440821FDF76AF999
:1053A0001E4BD4F8500102222421FDF763F994F832
:1053B0006C21D4F858011A4BB4F86011013A92B23A
:1053C000FDF758F91448FDF779F940B9404080F3EA
:1053D00011884FF0040002DFC4F80C21CCE7114A19
:1053E000111FFDF7B0F994F8293043F0380384F821
:1053F00029304FF6FF73A4F81A31A4F81C3142F299
:105400001F53A4F81E31BDE81040FFF75DBF00BF79
:105410001C020020440300205C03002070030020D5
:105420007803002064030020024B186843680021C1
:105430001B6818471C020020024B186843680021B3
:105440005B6818471C020020F0B4484003274FEA6D
:10545000102C082600240CF00105013E45EA440505
:1054600016F0FF06ECB24FEA5C0CF4D125022DB227
:10547000C0B24FF0080C344600F0010646EA44047E
:105480000CF1FF3616F0FF0CE4B24FEA5000F3D1F6
:105490002C4304EB0414013F0C4417F0FF07A0B2A7
:1054A000D5D125244140B1FBF4F004FB1010C0B26B
:1054B000C40800F00705145D2C41E40705D45943E6
:1054C000090C1046F0BCFEF7D3BEF0BC70470000DC
:1054D00070B514460E460546FEF7ACF82146FEF7B9
:1054E000ABF8C41C092C11D9094B1B7813B100204F
:1054F000FFF7D0F9324600212846FFF79BFDAB6845
:105500001C44262C00D8AC60012000E0002070BDB7
:1055100024040020294BDA7C70B502F0FF01054617
:105520001C462AB1404080F311884FF0040002DF8E
:105530001B7CDBB2052BF5D1A06094F82900012675
:1055400000F00700E67421746374FFF797FD94F888
:10555000293094F82820C3F3C20363F3020284F8CD
:105560002820FFF75DFB94F8293013F0C00F07D017
:10557000304602F0DFFF821C4178007803F026FB02
:10558000E26805F10901012003F076FB03F046FC17
:105590002A4605210A48FFF79BFF034628B104234A
:1055A0002375BDE8704003F071BA064A0146FDF765
:1055B000F1FF30F00203B5D170BD00BF1C02002026
:1055C000340200204148000010B5044603F0AAF957
:1055D000002003F0D1F90A4803F06EF904F110003D
:1055E00003F0E8F9637DA17D1B0243EA0143217DBD
:1055F00040F25B601943BDE8104003F083BA00BF7E
:10560000E95F00002DE9F8431C46584BDA7C074659
:1056100002F0FF061D462AB1404080F311884FF08A
:10562000040002DF1A7C238CD2B207339A42F3D1F2
:105630000323EB74A5F8186101232B75238DC5F89E
:105640001441D2B26385A860268520462E746A7400
:10565000FFF7BAFF962003F003FB3346324631468C
:10566000304603F079FA95F83921D5F8343153F8FA
:10567000221020460831FFF779F9637F580604F1BC
:1056800017024AD5608CE18B013803F03F0380B2EA
:10569000FFF7DAFEFFF7A4FAD4E91123134400223E
:1056A0006264226CA364934288BFA264D4E913238A
:1056B000002613442365EA68E66407F109013046D1
:1056C00003F0DAFA804603F075FB304603F094FBF2
:1056D000236DA26C78333146304603EB420903F068
:1056E000C2F9C84431468044304603F0BEF9404414
:1056F00003F042FB94F8201007313A46C9B2204625
:10570000FFF7E6FE034640B304232B7503F0BEF912
:105710000220BDE8F843FFF76FB9618DA67F01FB5A
:105720000666E17F25200E4496FBF0F100FB116632
:10573000F0B2C108E077515C06F0070641FA06F6C0
:10574000F10703F03F03A5D4B0FBF3F103FB110114
:10575000C9B21046FEF78CFD9CE7054A0146FDF7ED
:1057600019FF30F002037FF457AFD1E71C0200208D
:105770004148000010B590F8A840D0F8F02014F08F
:10578000800F18D1D0F8EC30ABB1240713D4D0F887
:10579000F840A34204BF1C68C0F8F84092B91A68E8
:1057A0000A601960C0F8F010C0F8F4100B680BB96B
:1057B000C0F8FC1010BD2AB9D0F8EC300B60C0F86E
:1057C000EC10EFE7D0F8F4301A680A601960EBE7E4
:1057D00010B490F8A84024070A460FD5D0F8F0106E
:1057E00031B9D0F8EC101160C0F8EC2010BC704753
:1057F000D0F8F430196811601A60F7E710BCFFF7B1
:10580000B9BF0000F8B5214F054607F5AA700E464E
:10581000FCF754FF0446B0B333797179D7F81421FB
:1058200043F07F4343F47E0343F4435343F01003B8
:1058300043EA0123B17943EA0143D2F88C10C1F362
:1058400010010B40C2F88C3092F8383043F020033E
:1058500082F83830037943F00303037108220923E7
:105860004371C37100211044FCF782FAD5F88C30E3
:1058700023721A0A1B0C28466272A3722146FFF794
:10588000A7FF0020F8BD0120FCE700BF1C0200209C
:105890002DE9F04F6F4D1C462B7C8FB0804689461A
:1058A0002BB1404080F311884FF0040002DF94F8E0
:1058B00020300733DBB22B7494F91D30002B09DA4A
:1058C000E36B616C02FB03330B44216C63648B421A
:1058D00088BF6164268D94F85C303244668C92B245
:1058E0002285324496B294F85D209A4271D0052008
:1058F000FFF7EEFB94F85E30013B032BD1D8DFE8D5
:1059000013F004002E027002B902D5F880310BB9F1
:10591000C5F8804194F8603013F0030300F0A680CE
:105920004D48FCF7CBFE0546002852D094F8603075
:1059300003F00302012AB4D16FF3010384F860304D
:10594000E38C0279063333449BB242F00302A4F89D
:10595000683002710C2242710022C27194F87020EA
:10596000027240F2E241E26EB2FBF1F2A0F80920CD
:10597000B4F86220A0F80B20B4F86420A0F80D2041
:10598000B4F86620A0F80F202268A0F81130002A91
:10599000C4F878800ADAD4E9011322F000428B427D
:1059A0002CBF434408EB01039B1AA36705F10903CD
:1059B0002A4A63672A4BC3E90242012211460020AA
:1059C000FCF732FF00287FF46CAF29462046FFF732
:1059D000D1FE94F8992094F898309A421DD0052071
:1059E000FFF776FB1C48FCF769FE0146A8B194F866
:1059F000983084F89930037943F00303037102234C
:105A00004371C37194F89A3003722046FFF7B2FED7
:105A1000E38D012B98BF0133A38694F8203094F9CD
:105A20001D5010481049A268073331EA250128BFEC
:105A30000146DBB2CDE90023CDE90214231D224645
:105A4000494640460136FFF751FB66840FB0BDE87A
:105A5000F08F00BF1C02002070030020454D0000A5
:105A6000C02A002005560000F1760000B4F86870E6
:105A7000F71BBFB23804ACD494F85C2084F85D20E6
:105A8000D5F880212B74944208BFC5F88031A28CD0
:105A9000B4F862309A4214D1B4F86410E38C99429D
:105AA0000FD140F2E2435A43B4F8663042F210712B
:105AB00001FB0323013B93FBF2F3E28D9BB29A427D
:105AC00016D00220FEF7F0FB00283FF4EAAE238C4C
:105AD000C380082303710023C372B4F8623083814A
:105AE000B4F86430C381B4F866300382FFF7FCF980
:105AF000D4E90036002B09DAA06823F0004386427F
:105B00002CBFB04480442360A8EB0308A38CB4F8F6
:105B100062A0CD4913FB07F39BB2B3FBFAF21FFA65
:105B200082F91AFB09F080B2834280F0F980C01A32
:105B300040F223124FEAE07C424301FB0C23A0FB1E
:105B400001011944BEA3D3E90023FAF799FB20F021
:105B50007F4000EB08030C93238DDFF814B3DB1BAD
:105B60004B44238523689E4238BF1E46E36E0A934A
:105B700094F91D300D9640F2E248002B08FB0AF61E
:105B800080F2E080E36B626C03FB172795F820310D
:105B9000AE4A32F8135094F83830C3F3820332F827
:105BA000133094F870201D44754305F57425A84BF7
:105BB00008FB02F205F23F25B5FBF3F5730805FB80
:105BC00009F0963B0744E26400229F4294BF676459
:105BD0006364E5632364A265A0FB0B0198A3D3E98A
:105BE0000023FAF74DFB0C9B1B1A0C930A9BB3FB8B
:105BF000F8F008FB00F092A3D3E90023A0FB0B010F
:105C0000FAF73EFB751B20F07F47B4F86430E3845D
:105C1000B4F86630A4F824A042F2107202FB0363C9
:105C2000013BB3FBF6F3E3858A4B3344B3FBF6F653
:105C300094F86030668613F0040308BF23860121C0
:105C4000002003F0C7F90022012181461046FCF72D
:105C5000C3FD94F8202041F68523002107320093EC
:105C6000D2B27D4B0846FDF71DFC30F002087FF4F0
:105C700018AEA5FB0BAB72A3D3E9002350465946DF
:105C8000FAF7FEFA002320F07F42CDE90A230A99B1
:105C9000724A94F8206007234B430B9902FB0133AF
:105CA0000A99A1FB02121A4420F07F450846BAEB7C
:105CB000000011466BEB01014FF47A720023FAF7F2
:105CC000DFFAE3680D9A94F91DC065491A4413463A
:105CD000644A32EA2C0228BF0A4641F6952108910F
:105CE00007365D49F6B2CDE90432CDE90641CDE98A
:105CF0000208CDE900750C9B324641464046FDF74F
:105D00003DFB30F002007FF4CCADB9F1000F3FF461
:105D10009DAE012211460FB0BDE8F04FFCF75CBD0F
:105D20000AFB12321FFA82FBABFB010140F2231384
:105D300003FB0B1142A3D3E90023FAF7A1FAA8EB66
:105D4000000308E70A993EA3D3E90023A1FB0B0156
:105D5000FAF796FA20F07F40471C354655E794F84D
:105D600060300BB34048FCF7A9FC054600283FF41F
:105D700030AE002384F86030E38C06333344A4F85B
:105D80006630037943F00303037108234371012351
:105D9000C371052204F161010830FBF7BCFFB4F8C0
:105DA0006630A5F80D3010E6B4F86630F31A190421
:105DB0003FF50FAE94F85C3084F85D3004F11705C0
:105DC000052204F161012846FBF7A5FF05212846BD
:105DD000FCF70AFE637F60F30503637701232377F3
:105DE000F7E52148FCF76AFC054600283FF4F1ADD1
:105DF00094F85C3084F85D301C4BC4F88C30037927
:105E000043F0030303710923437194F91D30002B00
:105E1000B4BF0E2308230822C37100211044FBF7EE
:105E2000A7FFD4F88C302B721A0A1B0C6A72AB7263
:105E300029462046FFF79EFC638EA386C9E500BF76
:105E40008D49FD1A070000000054CE0960B700001C
:105E500040420F00FF596202A54700008D49FD1A1C
:105E6000195F00001D5F0000700300200C4001005E
:105E700000CA9A3B94F89030DA0724D42548FCF7FE
:105E80001DFC014600283FF4A4AD94F85C3084F872
:105E90005D3094F8903043F0010384F8903003793A
:105EA00043F003030371062343710C23C3710923D9
:105EB00003726FF00E034372052383724FF0FF33BA
:105EC000C3720373B5E79B077FF5EBAC94F85C30C6
:105ED00084F85D300220FEF7E7F900283FF4E1ACDA
:105EE000238CC38001230371037A43F003030372FD
:105EF000062343720C23C37294F891300373B4F8F1
:105F00009230A0F80D30B4F89430A0F80F30FEF7BE
:105F1000EBFF5EE570030020FFF7BABCFFF7B8BCEB
:105F2000F8B590F8A8301A0604460F4608D4D0F801
:105F3000EC502DB11B07D0F8F0C022D5654520D01C
:105F400094F8A83043F0800384F8A83002F0F0FD04
:105F50000378012262F3010300224270D4F8EC209E
:105F60000370DBB252B143F01003037003786FF398
:105F700047130370002383703860F8BD62F3041385
:105F8000F3E794F8013194F800112A1DD01811B9E3
:105F9000417884F8001123B1D15C012666F3010138
:105FA000D15494F80061F61AF6B24670D15C1B2EFB
:105FB0006FF30411D15405D91B214170D15C41F01C
:105FC0001001D154296819B1D15C41F01001D154AC
:105FD000BCF1000FCAD1D4F8F8309D4218BFC4E913
:105FE0003C55C3E7000000002DE9F04F8FB002F0F0
:105FF00075FDC6B23EB302F091FD5FFA80F802F083
:1060000011FEC4B202F018FE02F0C2FF02F0AEFFB1
:1060100002F0D2FDC5B202F04BFD02F013FE02F019
:10602000F9FD02F0A9FF02F0BFFD6E48037D834633
:10603000052B01F25082DFE813F05F0087000A00B1
:10604000AD08AD08AD0835463446B046E3E7012358
:10605000037502F0FBFE0446962002F001FE9BF859
:106060001330013BC334032B11D8DFE803F00224C3
:10607000484800231A461946184602F06DFD02F002
:106080005BFD02F0DDFC02F01FFD054628B140403B
:1060900080F311884FF0040002DF014602F0E5FCB6
:1060A00029460444284602F0DCFC201A02F064FE73
:1060B00002F0B4FE20E0002319461A46184602F00A
:1060C0004BFD9BF83921DBF8343153F822000830BE
:1060D00002F0B6FC02F0F8FC05460028D7D10146D4
:1060E00002F0C3FC29460444284602F0BAFC201AF8
:1060F00002F042FE02F048FD0FB0BDE8F08F002331
:106100001A461946184602F027FD9BF83921DBF89C
:106110003431DBF8140153F822100831FEF726FC65
:1061200002F0D2FC05460028B1D1014602F09DFCE8
:1061300029460444284602F094FC201A02F01CFE72
:106140000120FEF759FCD7E72EB903238BF8143052
:1061500002F09CFCD0E7C37C013B032B97D8DFE81F
:1061600013F004000B026D046D04B8F1000FECD0C5
:1061700002F0E2FC9BF878202A234FF0270919FB54
:106180000239027802F00F03032B07460BEB0905D7
:106190002AD143780C2B27D19BF82930590600D5FA
:1061A00014B31BF80930C3F38013B3EBD21F1BD118
:1061B000062207F10801A81CFBF79DFDA0B90323E7
:1061C0008BF8143002F0D2FC9BF8C800272303FBA5
:1061D00000B07A3002F03AFC02F076FC00288BD056
:1061E00055E700BF1C0200203B7803F00F03052B8E
:1061F000ABD17B78222BA8D11BF8093003F00F0319
:10620000012B40F0958139462846FEF787FA88B180
:106210003B781BF80920C3F38013B3EBD21F40F087
:1062200085810622B91C05F10800FBF764FDB0FA70
:1062300080F04009002888D09BF87A3133B19BF870
:1062400078319BF879219A427FF47FAFDBF8CC302C
:10625000002B3FF47AAF0420FEF726F8054600280D
:106260003FF473AF4FF0040A8BF814A002F00EFC59
:10627000DBF8CC40DBF808114FF000084FF48272D5
:106280002046CBF8CC80FCF74AFA0322208407F1A1
:10629000120104F11400FBF73EFD04F1100318464F
:1062A00004F11706524607F10E010A93FBF733FD7E
:1062B000052207F11E013046FBF72DFD0521304672
:1062C000FCF792FB627F0A9B60F30502627797F806
:1062D0002320C2F30402A2773A8BA28440F2E24662
:1062E0005643F97EBA7E42EA0122E28419465246BA
:1062F00004F15400FBF70FFDBB8B42F2107202FB5E
:106300000363013BB3FBF6F3E385934B3946334418
:10631000B3FBF6F36386238C85F80B804FF00108FE
:1063200085F80C80EB8011F8023B0622C3F3801342
:106330002A716B7305F10E00FBF7EDFC3B8BAB8212
:106340007B8BEB82BB8B2B8397F82330C3F34213F9
:10635000AB76208CFEF706FAFEF7C6FD0320FDF7AC
:10636000A3FF00283FF493AE238CC3800A2303715C
:106370003B7813F0200300F0E980627C237CE17C11
:1063800043EA0223A27C42EA0122617F534041F0AA
:1063900040016177E38380F80B80FEF7A5FD97F855
:1063A000232094F838306D49520962F3840384F84D
:1063B00038309BF8203131F8122031F81330134473
:1063C000734303F57423664A03F23F23B3FBF2F3EE
:1063D000E3637308963B23647B7D40F2E24A4FF00F
:1063E00000080AFB03F323654146C4F84C8040468D
:1063F00002F039FB5B490A9000F2524054A3D3E902
:106400000023A0FB0101F9F73BFFDBF87C5165603D
:1064100027239D4238BF1D4620F07F402360E36B59
:10642000E060C4F80880F61A02F00AFD0B90F88AC2
:1064300041460AFB00AA404602F013FB0B9BAAF15F
:10644000300A9A440A9BAAEB000AAAEB03030A93B8
:1064500040F2834300930522434BDFF808A14146F5
:106460004046FDF71FF840F28441FEF7A1F91BF802
:10647000093003F00F03012B07D1CDF8008043460C
:10648000032241464046FDF70DF8A6FB0A6730A3FC
:10649000D3E9002330463946F9F7F2FEDBF808303D
:1064A000324AA3EB050B94F820300733DBB20B9391
:1064B00040F29B4308932E4BCDE906432D4B0593A9
:1064C000E36880461D4420F07F40072300214343BA
:1064D00002FB0133A0FB02121A440846301A11468F
:1064E0004FF000044FF47A724FF0000367EB0101A4
:1064F00004950394F9F7C4FE0A99029028F07F43AB
:106500000193A1FB0A0112A3D3E90023F9F7B8FE16
:106510000B9A20F07F4000905B4621460846FCF72E
:106520002DFF30F002037FF4B2ADE5E5002081E6F7
:106530009BF82930DB0900D034B139462846FEF7F4
:10654000EDF800F0010075E62046FAE7C37224E793
:106550008D49FD1A07000000FF59620260B7000074
:1065600040420F0000CA9A3BB14700008D49FD1A16
:10657000A5470000195F0000B8F1000F00F01A8273
:1065800090F8E130C3F3001313B1002C00F0128235
:1065900000228DF834209BF83911DBF8342152F8B1
:1065A0002170DBF8002107F10804DAB19BF87A21A9
:1065B0002AB19BF878219BF87911914212D1002BD6
:1065C0005FD19BF8E1203B7AC2F38012C3F38013C2
:1065D0009A4207D1062207F10A01DF48FBF78BFB3D
:1065E00000284ED03B7A13F00F0302D0062B40F068
:1065F000EE819BF8E120120740F1D881DBF8002101
:10660000002A40F0D3812846FEF7E4FC0546002826
:1066100040F0D08102F090FA0378D049032262F36F
:10662000030303703A7ADBB2C2F3801262F3C7133A
:106630000C2242709BF8E120D20962F386130446D3
:10664000062200F8023BFBF766FB062207F10A016F
:1066500004F10800FBF75FFB9BF8E03043F0020316
:106660008BF8E030962002238BF8143002F0F8FA11
:10667000284602F065FA204602F0E8F902F0CEFB67
:10668000AAE53B7A13F00F0340F0748102F0D8FBC7
:10669000DBF8DC3000F21626B1480722A3FB00012C
:1066A00002FB0311A8A3D3E90023F9F7E9FDA0F544
:1066B0009670864296D20420FDF7F6FD82460028A9
:1066C00000F0788104260023DBF800418BF8146089
:1066D000CBF8003102F030FA0378A04903F0D00380
:1066E00043F0250303703A7ADBB2C2F3801262F3FF
:1066F000C713222242709BF8E120D20962F386136D
:106700000546062200F8023B05F10809FBF703FBEA
:10671000062207F10A014846FBF7FDFA324604F16A
:10672000100105F10E00FBF7F6FA032204F1140143
:1067300005F11200FBF7EFFA01236B75BBF8F4309B
:1067400040F2E2465E4302F07BFBDBF80C20DBF814
:106750000481002A00F5DB63D8BF00F2BA63B8F108
:10676000000F40F0138185F8168085F81780984651
:106770000021084602F070F90021A8EB0008084645
:1067800002F06FF9A8EB000000F11E030A93BBF8BA
:10679000F4302B83BBF8F6306B83BBF8F830AB8357
:1067A00004F11701052205F11E00FBF7B4FAA27FE0
:1067B00095F8233062F3040385F823309BF82021F9
:1067C00062F3471385F8233002F0D0F9284602F02F
:1067D0003DF902F079F9804600287FF458AC4FF477
:1067E0008272DBF808112046FBF799FF20848AF8B3
:1067F0000B808AF80C802B78AAF806000622C3F3D7
:10680000C0138AF8042049468AF80D300AF10E00B8
:10681000FBF781FABBF8F430AAF81430BBF8F63075
:10682000AAF81630BBF8F830AAF8183095F82330DB
:10683000C3F342138AF81A30208CFDF793FFFEF75A
:1068400053FB0320FDF730FD00283FF420AC238CE0
:10685000C3800A2303713B7A13F020030ED0627CBD
:10686000237CE17C43EA0223A27C42EA0122617F8D
:10687000534041F04001E38361770123C372FEF787
:1068800033FBDBF87C316360272B38BF27232722BB
:10689000002522609846DBF8FC20E2604FF4C763D5
:1068A0000622A5602946009328462E4BDFF8C0A09B
:1068B000FCF7F8FD40F23961FDF792FF2B46042208
:1068C000294600952846FCF7EDFDDBF8083094F8E2
:1068D0002090A3EB080B4FF4CA630893224BCDE939
:1068E0000643224B0593E368A6FB0A674344CDE9C0
:1068F0000353304616A3D3E900233946F9F7C0FC09
:10690000104619464FF47A720023F9F7B9FC10A328
:10691000D3E90023029039463046F9F7B1FC0A99D1
:1069200001900BA3D3E90023A1FB0A01F9F7A8FC0E
:1069300009F107095FFA89F920F07F4000905B4672
:106940004A462946EAE500BF00CA9A3B000000001B
:106950008D49FD1A0700000004030020FE020020FC
:106960008D49FD1AE1470000A54700001D5F0000AA
:1069700000CA9A3B012B7FF435AE00212046FEF77A
:1069800083FA00287FF482AE2CE6B044B8F1000F01
:10699000FBDB9845F9D3A8EB030340F2E242B3FBDB
:1069A000F2F3EB826B7D01336B75E1E67BB97B7AA9
:1069B000002B3BD103238BF8143002F067F89BF8CF
:1069C000E0306FF341038BF8E030FFF795BB012B0C
:1069D0000DD03B7A03F00B02022AE8D003F00F033C
:1069E000072B0BD19BF8E1305B07E0D1E2E70DA963
:1069F0002046FEF749FA0028D9D1EAE7042BD9D17D
:106A00009BF8E0309E07D5D502F096F83B7A0278E5
:106A1000C3F38013B3EBD21FCCD1062207F10A01D6
:106A20000830FBF768F90028C1D0C3E7DBF8003174
:106A3000002BBFD12846FEF7CDFABBE790F81831FE
:106A400090F83921013380F81831D0F8343153F8F7
:106A5000226001233371D0F81431B8F1000F00F037
:106A60002C8393F8A820307A02F00101C0F3800053
:106A7000884200F0A88081F0010161F3000283F8F0
:106A8000A8209BF81320032A02BF93F8382042F075
:106A9000010283F8382093F8A820140600F18F80B3
:106AA000D3F8EC7093F801C107F1040E0EEB0C055E
:106AB0006C780CB9002528E090060BD5D3F8DA9055
:106AC000D3F8DEA019F101004AF10001C3F8DA00A1
:106AD000C3F8DE101EF80C3003F00303032BE9D1DA
:106AE000EA78022AE6D18BF8143001F0CFFF01F0EA
:106AF000EBFF00287FF4CBAA2979DBF814011329D6
:106B000008BF1621FEF738FA0125DBF8142192F8A8
:106B1000013192F800112344DBB2994282F801312D
:106B20002AD00027002D4FD0DBF81401FDF7B4FF69
:106B30000025CBF8145102F065F918B902F056F9A6
:106B400002F05AF9DBF81431002B3FF4D5AA1FB13B
:106B50003946188CFDF72CFF002D3FF4CDAADBF849
:106B60001431188CFDF7FEFDDBF814311B8CF3801B
:106B7000FEF7BAF9FFF7C0BAD2E93B3100208B42E9
:106B8000A2F8000111D1002FCBD0D2F8F4101C686C
:106B9000C2F8EC408B420CBFC2E93C00C2F8F040A6
:106BA000C3493846FBF7A3FDBBE7D2F8F8101868D5
:106BB000C2F8EC008B4208BFC2F8F800B2E76FF3EE
:106BC000C71283F8A8200027DBF81431327A93F833
:106BD000A830C2F3C002C3F340039A4240F08F8151
:106BE0000320FDF761FB002800F089819BF87A31D2
:106BF00083B3DBF84431DBF84821934205D19BF89D
:106C000078219BF87911914224D0DBF848219342F6
:106C100000F075819BF878319BF879219A4200F059
:106C20006E819BF87831DBF8142123B9BBF876111B
:106C3000138C99420ED09BF87831002B00F05F81C5
:106C40009BF878310BEB4303B3F87011138C994226
:106C500040F0558196F80990B9F1000F00F03181AC
:106C6000DBF8143193F8A89019F0100906D002F05F
:106C700055F900283FF40BAA4FF00109DBF8143155
:106C800093F8A830D9060FD4DBF81441337A94F87E
:106C9000A82012F0040F20D113F0030300F011819B
:106CA000022B47D80125B3E002F056F90028EBD1BA
:106CB00003238BF8143001F0E9FE01F005FF0546CF
:106CC00000287FF4E4A9DBF814013D21FEF754F914
:106CD000DBF81401FDF7E0FE2BE703F003010329C5
:106CE000E6D194F91D00F17A002802F0400215DB8C
:106CF00022B90229D0D01129DAD809E08A1ED2B2ED
:106D0000092AF8D840F2052020FA02F2D207C3D4AB
:106D1000684A22FA01F1CD07CAD5BDE72AB902298E
:106D2000BAD01129C4D8644AF3E78A1E012AB3D91C
:106D30000B29F5E7F57A06F1080A192D00F27A8198
:106D4000DFE815F01A008400C100780178017801AD
:106D500078018C01CA00E700780178010D01780103
:106D6000DF007801780171017801780178017801FC
:106D7000780178017801930194F91D30002B80F29D
:106D80005981717A0020FDF747FA002800F05281FE
:106D9000B6F81510638CCB1A180400F18F8094F8A4
:106DA0005C3094F85D209A427FF471A9DBF8802171
:106DB0000AB9CBF88041327B84F87020B6F80D0018
:106DC00040F2E2424243E266307CF27B42EA002239
:106DD000A4F86220B07C727C42EA0022A4F864200D
:106DE000F27C307DA4F8681042EA0022A4F8662004
:106DF00094F8602002F0FC026FF3820284F86020B5
:106E0000013B0122002584F85E2084F85D30A586D0
:106E1000DBF8141191F8A83083F0020381F8A83050
:106E2000B9F1000F0BD0D1F8B990D1F8BDA019F18C
:106E300001024AF10003C1F8B920C1F8BD30DBF806
:106E4000143100248BF819411C864BE194F91D3054
:106E5000002B80F2EF80717A0120FDF7DDF9002828
:106E600000F0E880628CB6F811309B1A1A0425D421
:106E700094F85C2094F85D309A427FF408A90522CA
:106E800006F10C0104F16100FAF745FF737CB27C56
:106E900043EA0223A4F86630022384F85E3094F8B3
:106EA0005D300025013B84F8605084F85D30AFE729
:106EB000700300206020020040200200282384F894
:106EC0009B300025A4E7717A0220FDF7A5F9002880
:106ED00000F0B080337BF2E794F91D30002B80F294
:106EE000A980717A0820FDF797F9002800F0A280A8
:106EF00051462046FEF786FC0546002888D000252E
:106F00009DE794F91D30002BC0F29480717A0E2019
:106F1000E9E7717A0920FDF77FF9002800F08A80FF
:106F2000337B727B43F07F4343F47E0343F443534C
:106F300043F0100343EA0223B27B43EA0243D4F84E
:106F40008C20C2F310021340C4F88C3094F838300F
:106F500043F0200384F838300023A386A2E6717A38
:106F60000C20FDF759F9002864D094F8903013F004
:106F7000010551D1C448FBF7A1FB01460028BED052
:106F800094F8903043F0010384F89030037943F093
:106F900003030371062343710C23C3710923037296
:106FA0006FF00E034372052383724FF0FF33C372F9
:106FB00003732046FEF70CFC94F8A83043F08003DE
:106FC00084F8A83001F0B4FD03784570012262F323
:106FD0000103D4F8EC200370DBB2C2B143F010031C
:106FE0000370337B84F89130B27B737B43EA0223D6
:106FF000A4F89230F37B327C43EA0223A4F8943065
:1070000094F8903043F0020384F8903000E762F384
:10701000041303701546E4E713F002037FF451AF45
:10702000A3860125DDE7717A1120FDF7F5F8002828
:107030007FF447AF9448FBF741FB014600283FF43B
:107040005EAF0379057243F00303037102234371BA
:107050000723C3712046FEF78DFB32E7717A0720C4
:10706000FDF7DAF80028E5D076E794F91D30002B1B
:10707000E0DB717A1920FDF7CFF80028DAD0357BF4
:1070800015F001053FF4C4AE94F85C2094F85D302F
:107090009A427FF416AF05227C4904F16100FAF7A9
:1070A0003AFE012384F86030022384F85E3094F8BD
:1070B0005D30013B84F85D3003E790F8192112B987
:1070C000022280F819219BF81941013CE4B28BF8A7
:1070D00019411D8EB4FA84F46409002D43D1DA8D70
:1070E0001A862F46DBF814010DA990F8A890FEF738
:1070F00017FF9BF81430032B4FEAD91938D0A4BBE3
:10710000B8F1000F05D0337ADB0602D40D9B5B7813
:107110005BB3DBF8143193F89B4034BB0223962019
:107120008BF8143001F09CFD204601F009FD01F0C0
:1071300075FEDBF814010D9990F8A8200B78C2F3C6
:10714000000262F3C30390F8A820C2F3400262F386
:1071500082030B70FDF724FD01F0B6FC00283FF41C
:10716000EAACFEF794BF0025BBE703238BF814308D
:107170009BF81330042B0AD1DBF8143193F8A820C4
:1071800069F3C71283F8A82001F080FCD3E401F072
:10719000EDFCCEE7C27C042A3EF679AFDFE812F0C0
:1071A000930105005200A900A900032B09D190F812
:1071B00028305D0705D0FDF733FD01F061FCFEF7D7
:1071C00077BF01F01DFD9BF81430032B71D19BF8A4
:1071D000284014F040046CD101220DA9DBF8040012
:1071E00002F090FE9DF8341029480A23B1FBF3F217
:1071F00003FB12120132D2B2D5B2A5FB0001E82383
:107200008DF8342003FB05111DA3D3E90023F9F702
:1072100037F840F64B7306931E4BCDE90244CDE997
:107220000443CDE9004483B2052221462046FCF701
:10723000EFF830F002033CD09BF81230052B38D029
:10724000FEF725BF032B27D1962001F009FD00236F
:1072500019461A46184601F07FFCDBF834319BF8DA
:10726000392153F82200083001F0EAFB01F08CFCD0
:1072700001238BF8143001F0FDFBFEF719BF00BFAE
:107280008D49FD1A0700000070030020360300201E
:107290000010A5D41148000001F0B2FC9BF8143096
:1072A000052B06D100230093042219461846FCF74B
:1072B000F9F800248BF813408BF814408BF8114038
:1072C00001F04EFD224621462046874BFBF7ACFAE3
:1072D000044600287EF4DBAEDBF80000436821465C
:1072E0005B689847012211462046FBF775FAFEF7C6
:1072F00003BFD0F814010028DBD090F89B1089B1AF
:107300009BF81330032B03D090F83830DC0709D5F5
:10731000FDF732FEDBF81401FDF7BEFB0023CBF8CE
:107320001431C6E7468D9BF81871751CADB2002F5D
:107330006BD09BF81330032B5BD101F063FD8046CB
:1073400001F066FDDBF81471DFF8A491A8EB0008EA
:10735000B86C00F1580AD04561A3D3E900233BD8AB
:10736000A0FB0901F8F78CFF84B2AAEB08005CA32C
:10737000D3E90023A0FB0901F8F782FF83B20022C2
:10738000BA643A65D7F8EC206AB3527912B997F823
:1073900001210AB100227A85DBF8142100219185B0
:1073A000DBF81401028EAAB1954280F08480521B52
:1073B00092B20021062A028641857ED99BF81320CD
:1073C000032A07D1002E78D1476D7A0817F00107FC
:1073D00035D14265002735E0A8FB0901F8F750FFD9
:1073E000022384B2CBE797F83820D207D4D5FA8CA1
:1073F000D1E741B190F8383043F0010380F83830DC
:1074000000231C46C8E70B46FBE7848D84B1A542E8
:1074100004D2641B84853C462346C1E73E21FDF728
:10742000ABFDDBF81401FDF737FBCBF8147140E737
:10743000038E002BF0D1C28D02861C46B0E742F0CD
:1074400000424265828E1AB1954238D2551B85861C
:1074500090F85D1090F85C20914206D090F85E2084
:10746000013A012A9CBF00224285418D0FB98E420C
:1074700027D0013189B224B91BB911B9002F3FF4CB
:1074800018AF90F82050194A039107350021EDB24A
:10749000CDE90472009306952346CDE901112A46F1
:1074A0000846FBF7B5FF30F002033FF402AF9BF84C
:1074B00012309D42C3E608212AE70127C2E72221B4
:1074C00026E73946D7E7043B012B3EF6E0AD002323
:1074D0000375FEF711BEFDF777FD00BFAFF3008027
:1074E0008D49FD1A07000000602A0020294800008D
:1074F00000CA9A3B000000002DE9F0418EB0022343
:1075000009930023CDE90A33FF22734E734D8DF8A2
:10751000232004460C9309ABCDE901630CAB009327
:107520000DF123020DAB01210020FBF7F5FF02282E
:107530000BD0099B6BB1404080F311884FF00400E1
:1075400002DF01210020FCF75FF8099B022BF8D035
:10755000EFE79DF82330FF2B04D095F81021073278
:107560009342D8DA5A1FD2B2F92A5D4F05D85B4A46
:1075700092F810210732934207DB3B7813B10120C8
:10758000FDF788F90EB0BDE8F0810AA9E0B2FDF779
:1075900063F90028CFD0D0E90034002BB8BF83684E
:1075A0009C4238BF1C46C3689DF823000BA91C44AD
:1075B000FDF752F905460028BDD0D0E90136026832
:1075C0009E4238BF1E46002A05DA0C9B22F000427C
:1075D00033449B1A0C930C993A7804F131038B4293
:1075E0000AD212B10120FDF755F99DF8232001219F
:1075F0002846FDF71FFDC5E73AB90120394B387021
:107600001146FBF711F9002895D12B68002B15DBEB
:10761000B34213D99B1B00209BB233490591CDE99E
:1076200001039DF823200695CDE903000090012178
:10763000FBF7EEFE30F002037FF47DAF0A9E002ED2
:10764000A0D00B9D002D9DD0B38CAA8C9A4299D1CD
:10765000264897B2A7FB000140F2231303FB071152
:107660001BA3D3E90023F8F70BFE0C9B20F07F400F
:107670000022834218D802B10C9396F91D1095F997
:107680001D20002913DA002AFFF67CAF1434A34230
:10769000BFF478AF3046FCF723FE02287FF472AFC8
:1076A0000B98FCF71DFE6DE71B1A0122E1E7002A8B
:1076B000BFF668AF1434A342BFF464AF2846FCF7AA
:1076C0000FFE02287FF45EAF0A98EAE7AFF300806E
:1076D0008D49FD1A07000000554200001C020020E1
:1076E00024040020E02A0020594200000054CE0962
:1076F000F7B51C46494BDA7C074602F0FF061D46EB
:107700002AB1404080F311884FF0040002DF1B7C57
:10771000228CDBB207329342F3D10422A5F8186120
:10772000DBB2EA742E746B74238DC5F81441022009
:10773000638526852875AF60FDF75EF901A92046AF
:10774000FEF7EEFB019994F8A8200B78C2F3000233
:1077500062F3C30394F8A820C2F3400262F38203E9
:107760000B702046FDF730FF962001F079FA304685
:1077700001F0E6F920460199FDF712FA637F5806F9
:1077800004F1170221D5608CE18B013803F03F032F
:1077900080B2FDF759FEFDF723FAEA6807F1090107
:1077A000012001F069FA01F039FB94F8201007314B
:1077B0003A46C9B22046FDF78BFE034628B30423A0
:1077C0002B7501F063F903B0F0BD618DA67F01FB5D
:1077D0000666E17F25200E4496FBF0F100FB116662
:1077E000F0B2C108E077515C06F0070641FA06F6F0
:1077F000F10703F03F03CED4B0FBF3F103FB11011B
:10780000C9B21046FCF734FDC5E7054A0146FBF74F
:10781000C1FE30F002037FF474AFD4E71C020020F5
:10782000414800002DE9F0413C4E0A9C9DF81C8027
:10783000BDF82C50BDF820E09DF818C030604FF422
:10784000827000FB034086F82011C6F808416119D8
:1078500008F10104E7B272600EF103040CF10302B7
:10786000282CD2B2A6F82CE186F84C2188BF0EF164
:107870000E0E92B294BF02EB42022EF0030E0CF1F8
:10788000040C08F102085FFA8CFC8CBF1EFB02F2AC
:1078900012015FFA88F8A6F82E2186F86C81C6F8E6
:1078A00034014FEAC80800EB8C00B6F82E41C6F848
:1078B000640140443022C6F868014044A6F83021F3
:1078C000C6F82401B4FBF2F220440CEB0304C6F822
:1078D0003C0100EBC400BDF82440C6F850010A3456
:1078E00024F003044830A4B2A6F8604107FB040466
:1078F000641A86F8103186F838C186F83221C6F845
:10790000580103D02C442046BDE8F081012386F8BD
:107910007A31FDF723FD00F0E3FFF4E71C020020BD
:1079200038B503210520FCF76FFD04210620FCF784
:107930006BFD214C002594F81021ABB29A4205F161
:10794000010532D894F828306FF3C71384F8283033
:1079500094F8E030002060F3000384F8E030302237
:10796000B4F82E31B3FBF2F384F8323194F83831A5
:1079700084F83901013B84F86D0184F8700184F8C2
:107980004C3194F87831C4F8CC00C4F80001A4F864
:10799000302184F83A01A4F86E0184F8793100F0BE
:1079A0006BFEBDE83840FDF7D9BCA81DFF21C0B271
:1079B000FCF72AFDBFE700BF1C0200200520FDF7F1
:1079C00087BB00000048704746020020004870470F
:1079D00096020020024B93F82800C009704700BFB0
:1079E0001C020020044B93F92820002ABABF93F808
:1079F00029008009002070471C020020094A92F8E3
:107A0000E03092F8E100D2F80021C0F3C000002A73
:107A100003F0010303FA00F314BF0420002018430D
:107A2000704700BF1C020020054B93F8E00010F0E7
:107A300001001CBF93F8E100C0F30110704700BFC4
:107A40001C02002010B51446FCF7C8FC10B1002041
:107A5000207010BD0120FCE72DE9F34105460846E2
:107A60001849D1F84431D1F8482193420F461FD02C
:107A7000D3F8048001F26F1198F80020FCF764FC41
:107A80000446E0B902AE97F86F3106F8033D97F867
:107A9000702131460DF10600FCF756FC34B928B9C7
:107AA000C5F80080204602B0BDE8F0810446EEE74C
:107AB00091F8702101F26F11FCF746FC0446002397
:107AC0002B60EFE71C0200202DE9F041164C054623
:107AD0000068A4F59476A4F11C0720B92860BDE8DD
:107AE000F041FDF7F1BB0279D0F800800A2A07D8EF
:107AF0000123934040F27E72134207D11B060AD441
:107B0000404080F311884FF0040002DF2146FAF76D
:107B1000EEFD4046E1E7C288D6F808014FF48271D5
:107B2000FAF7FAFD3946F2E744030020914210B516
:107B3000144B19D1D3F84821D3F84441944211D1C0
:107B4000002914BF0A460322013AD2B203EB4204D1
:107B500083F8792193F87821A4F8720191420FD02B
:107B600083F87911012005E029B9B3F87631181AA4
:107B700018BF012010BD03EB4103B3F87031F6E7E5
:107B80000020F7E71C02002030B4144B93F87A2150
:107B90000D4602B393F87821D1B293F8792135B12B
:107BA0004FF6FF73984216D030BCFFF7BFBFD3F833
:107BB0004401D3F84841A0420DD191420BD0D3F8F3
:107BC000484183F87911A04205D093F878018842A2
:107BD00008BF83F87921002030BC70471C020020C8
:107BE00070470000000000002DE9F04FA04F8FB05B
:107BF0009A4602230D9397F928308DF82F20002BF9
:107C0000834688463D4601DA0C202AE197F8792020
:107C10002A234FF0270919FB023917F8093003F01E
:107C20000F03012B00F2D680D7F8CC60002EEBD1E9
:107C300007F5A070FAF742FD0A9058B107F5867073
:107C4000FAF73CFD0A9A044630B907F5A0711046D0
:107C5000FAF74DFD072004E14FF6FF730384854BCF
:107C6000C0F88C30437FC67766F3861363F07F03DA
:107C700043770623838590F83830468466F34513AE
:107C800066F3000366F3410380F8383090F89030D3
:107C9000866266F30003C0E93B66C0E93D6666F3B1
:107CA0004103C0E91166068686868665A0F85C6099
:107CB00080F89030A0F8986080F89B60C0F89C2015
:107CC00080F8A860C0F8FC60A0F80061C7F8CC009C
:107CD0000EA895F8293010F8092D6BF3020362F312
:107CE000C5036AF3871385F82930D5F87C31EB6139
:107CF0002723AB61012100232B62FAF775FE17F8E9
:107D0000096006F00F06012E66D14FF42773584321
:107D100000F59C70584954A3D3E90023A0FB01014E
:107D2000F8F7AEFAD5E906739F42686238BF1F467E
:107D3000B8F1000F58D1721E5342534195F8286094
:107D4000DFF84891DFF848B163F3861685F82860BC
:107D500016F040060DF1340A4ED0FBF76BFC6B6A4F
:107D600006461F440020CDE9079ACDE905B0CDE9CC
:107D70000307CDE901700090334605220321FBF78C
:107D8000FDFA022834D00D98B8B902230D933B4B6D
:107D90000690CDE9079ACDE90200CDE9040303225C
:107DA0004AF2FE330093019033461146FBF7E6FAA0
:107DB000022843D00D98002844D0002C3FF424AF73
:107DC000D4F89C002E49FAF792FC2E492046FAF787
:107DD0008EFC19E700247BE7022E0CBF4FF42973B9
:107DE00040F2FC53584395E70023A7E7FCF710FA4D
:107DF0000D9B022BFAD0C6E7FBF71CFCCDE9079AD6
:107E0000CDE905B60A906B6A1F4802961FFA88F8FA
:107E10001F44A8FB0001912303FB081112A3D3E91F
:107E20000023CDE90367F8F72BFA0A9BCDE9006040
:107E3000052203213046B9E7FCF7EAF90D9B022B36
:107E4000FAD0B7E795F8283043F0800385F828305A
:107E500095F8E03013F0010403D10120FFF7C0FED4
:107E600020460FB0BDE8F08F8D49FD1A07000000D5
:107E70001C0200200C40010000CA9A3B99520000ED
:107E80005C03002028030020002AE78455420000FC
:107E90006152000070B503210520FCF7B5FA0546D4
:107EA000E8B9104C94F8282060F3C71284F8282011
:107EB00094F8E020D30701D4FFF792FED4F8CC6009
:107EC0005EB100230849D6F89C00C4F8CC30FAF71C
:107ED0000EFC06493046FAF70AFC284670BD0C2510
:107EE000FBE700BF1C0200205C03002028030020E9
:107EF00037B5344D02AA002342F8043DD5F84801B5
:107F000005F5A271FAF731FC2C4628B9404080F300
:107F100011884FF0040002DF05F5A071FAF7E7FBC6
:107F2000019A11790A29F1D801238B4040F27E7021
:107F3000034211D11806E9D5062935D1D37A3C2B55
:107F400015D0127B92BB94F8E030D907DED562F3EE
:107F5000000384F8E0301AE095F8380195F84C31C8
:107F600001388342D2DA013385F84C31E4E700234B
:107F7000D4F8CC50C4F8CC3094F92830002BC5DAB2
:107F800094F828306FF3C71384F8283085B994F833
:107F9000E00000F0010394F82800C0F3C01050EA9C
:107FA000430001D1FFF71CFE03B030BD0025E3E71D
:107FB000D5F89C000449FAF79AFB04492846FAF7D9
:107FC00096FBE4E71C0200205C030020280300204D
:107FD00038B50B4CD4F84021D4F8445122B10020DC
:107FE000C4F84001FBF7B8F92DB10023C4F84431BF
:107FF0000120FBF7B1F90020BDE83840FAF762BC78
:1080000000B000400120FAF75DBC684620F007018F
:108010008D4601B500F048FCF9F704FDF9F7EEFADA
:10802000BDE801408546704770470000014B186865
:1080300002F091BC180A002070B5384B86B0186069
:10804000374801F07BFF18B96FF0120006B070BD21
:10805000436801211B689847324801F06FFF0446CE
:108060000028F1D000F014FBFAF78CFB2E4B032212
:108070001A721A76082100202C4A19701874059279
:108080002B4A04922B4A03922B4A02920E22CDE9EC
:1080900000320423294AFBF717F9064628B140406D
:1080A00080F311884FF0040002DF254801F046FFFD
:1080B0000028C9D04FF4F8730593224B04931B2377
:1080C000CDE9023301250223CDE900532246334690
:1080D0000721FFF7A7FB0446E0B9284600F0CCFAD9
:1080E000224621462846F9F783FC224621460B20EA
:1080F000F9F77EFC224621461820F9F779FC28463C
:10810000F9F744FC0B20F9F741FC1820F9F73EFC85
:1081100020469BE76FF00B0098E700BF180A00208D
:1081200068B2000044B20000F8090020D5900000B9
:108130005D9000003D9000005807002018060020C8
:1081400073B200002804002007230B700023037083
:10815000704700002DE9F04385B09946734B0293B8
:1081600040F201730D461446119E9DF84870ADF81B
:108170000C30FFF72FFC8046002840F0D1806C497E
:108180000B78012262F34713B9F1040F0B700BD97E
:10819000E80605F003030FD5664A01922A0706D4C4
:1081A00004AA134413F80C9CB9F1010F12D1002357
:1081B0004B604FF001090EE0032B00F0B48005F096
:1081C0000C030C2B00F0AF800B7867F347130B7098
:1081D0004FF005094C600B789DF83C2062F30203D8
:1081E0009DF8402062F3C4030B70FFF7EBFB90F89F
:1081F0004F2002EB8203C2EBC30204AB9944835CC1
:1082000019F8081C9DF8309061F303036FF3041311
:108210008354DBB203F00F01012994BF43F0200324
:108220006FF345138354835C09F0010969F38613E6
:108230006FF3C7138354DBB203F00F01012900EB86
:1082400002040DD19DF8341061F3C71383540E99C5
:10825000062204F10800F9F75EFD0C2363703CE090
:10826000072958D1A17801F0C00165F38711A170E9
:10827000A8064FF0000104F1020304F10402E170CA
:1082800009D4A17811F0C00F05D1042F1EBF01221F
:10829000E27004F10A02690644BFE1780132A2EB00
:1082A000030348BF41F04001DBB248BFE170022B3D
:1082B0008ABFA178012303F1FF306370E37884BFA4
:1082C00060F30501A1705B0607D516B333787F2BE9
:1082D00001D10023337002F8013CFFF777FB90F8DF
:1082E0004F2002EB8203C2EBC3020424835C64F3DD
:1082F000030303F0CF0369F386136FF3C7138118E9
:1083000083544B780BB906234B70404605B0BDE84B
:10831000F0833346DFE76378002BDED106239DE749
:108320004FF00C08F1E74FF01208EEE700010602EB
:108330001C0A0020030402002DE9F0410F46064606
:10834000FFF740FB90F84F5005EB8502C5EBC202EA
:10835000044610F802C00CF00F03012B00EB0201E1
:1083600040D0072B3ED090F84E30AB4204D10135BF
:10837000EDB2022D08BF002505EB8503C5EBC30355
:1083800004EB0308E05C6CF303006FF30410E054AB
:10839000A05C14F803C0C0F3401060F3451C04F85F
:1083A00003C0A05C5FFA8CFCC0F3801060F3861CF5
:1083B00004F803C0A25C5FFA8CF0D20962F3C71024
:1083C000E0540622023108F10200F9F7A4FC32461B
:1083D000394608F108000636F9F79DFC88F8016077
:1083E00084F84F50BDE8F0812DE9F04106460F4674
:1083F000FFF7ECFA90F84F3090F84E209A4204467E
:1084000036D15D1CEDB2022D08BF002503EB8302BF
:10841000C3EBC2022BB203EB8300C3EBC0034FF0EC
:10842000040CE05C6CF3030000F0EF006FF3451008
:10843000E054A05CA118E25CC0F3801060F38612E7
:1084400004EB03086FF3C712E254B31D88F8013040
:108450000622023108F10200F9F75DFC3246394686
:1084600008F10800F9F757FC84F84F50BDE8F08197
:108470001D46CBE72DE9F74320B903B0BDE8F04333
:10848000FFF708BDFFF7A6FA074600284ED1FFF711
:1084900099FA8046FFF79AFA98F84F4004EB840364
:1084A000C4EBC304064618F8040000F00F03072BC2
:1084B00008EB04091DD199F80330DB070AD53946CA
:1084C000C0F38010FBF7BCF80622014609F1040056
:1084D000F9F721FC164B18789988FF23009300F0D8
:1084E0000702C0F3C1034009FFF77EFB03B0BDE8FC
:1084F000F0833946C0F3801096F84F50FBF7A0F890
:108500000622014609F10200F9F705FC18F80400FB
:108510003946C0F38010FBF793F805EB8503C5EBF4
:10852000C305354401460622A81CD1E70020DDE73B
:108530001C0A002028B9404080F311884FF0040045
:1085400002DF0148704700BF240A0020082070475E
:1085500010B5FFF747FA044610B10C24204610BDB1
:10856000FFF762FAC307F8D4024B1C705C70024B31
:108570001C70F3E7240A0020900F002070B5044619
:10858000FFF730FA054610B10C25284670BDFFF7FD
:108590004BFAC307F8D42378FF2B03D1114B0122E8
:1085A0001A70F2E7611C104C2278FF2A17D0284677
:1085B00022FA00F6F60710D40126864032432270D4
:1085C00003F00103627883401343062202FB00405C
:1085D00002306370F9F79FFBD7E70130E8E7072522
:1085E000D3E700BF900F0020240A00202DE9F047B8
:1085F0000746FFF7F7F9064618B10C263046BDE8E6
:10860000F087FFF711FAC107F7D497F80080B8F1A7
:10861000FF0F02D1164B1E70F0E7164C23780BB9F2
:108620001226EBE7082501374FF0060904F1020A8C
:1086300015F1FF35F4D32378EB40DA07F8D56378EA
:108640002B4183EA0803DB07F2D40622394609FBF3
:1086500005A0F9F750FB0028EAD10123AB402278AE
:10866000DB43DBB21A402270627813406370C5E7C7
:10867000900F0020240A0020034A00231370034AAD
:1086800013705370704700BF900F0020240A002021
:10869000054B0022C3F808254FF44032C3F84423A9
:1086A000C3F80423704700BF00B00040044A1378A9
:1086B000591C1170012013B9024A10601846704706
:1086C000560A002000B00040094B187828B94040F5
:1086D00080F311884FF0040002DF0138C0B2187037
:1086E000012310B9034A136070471846704700BF52
:1086F000560A002004B00040014BD3F8040570472F
:1087000000B0004000F5A870014B43F820107047FE
:1087100000B00040F0B5134B134C012584462E46A3
:108720000027A6461A462660C3F804C5C3F80071A0
:10873000C3F804711E60D3F8001131B9D3F80411E5
:1087400019B9D3F804150029F5D1CEF80050D2F8A4
:1087500004110029E7D1D2F804050028E3D0C2F8BB
:108760000415F0BD00E0004004E0004070B58CB09E
:108770000E4615460146102268461C46F9F7D4FFFE
:1087800010220DEB02003146F9F7CEFF6846FFF7E5
:10879000C1FF25B1102208A92846F9F7C5FF24B169
:1087A000102208A92046F9F7B6FA0CB070BD0000F7
:1087B000094B0A4A002814BF1846104603F5F03347
:1087C00002F5E2423C32C3F810250122C3F8140539
:1087D000C3F80425704700BF00100040041000409B
:1087E000F0B52C4E2C4F35782C4BC7F860352BB29A
:1087F000DC0004F1804404F5F834C7F8644505F161
:108800000B04E4B2E400A7F5AF3704F18044C03FA5
:1088100004F5F83407EB8307C4F81075002834D04A
:1088200049F6404049F6C477022A0CBF02463A4650
:1088300041F2883042F2B847022918BF384602F5A3
:10884000FA7101444FF47A72B1FBF2F1144AC4F8A0
:1088500014259B0003F1804303F51043D3F8402512
:108860008A428BBFD3F840250122511AC3F8402514
:1088700088BFC3F84015084B4FF49062C3F8042535
:108880006B1C03F001033370F0BD064AC4F81425D5
:108890002C21DEE7740C002000F001400C11004098
:1088A0000010004004100040024B1B6803B1184741
:1088B000704700BF700C0020064B1860064B10225A
:1088C000C3F80423054B0222C3F880210120F9F7E5
:1088D0005DB800BF700C00200010004000E100E017
:1088E0004FF080434FF0FF320021C3F8002EC3F851
:1088F000042EC3F8081EC3F80C2EC3F8101EC3F8CC
:10890000142EC3F8182EC3F81C2EC3F8202EC3F85B
:10891000242EC3F8282EC3F82C2EC3F8302EC3F80B
:10892000342E704708B50120F9F740F8084B0022B3
:10893000C3F8FC2F0122C3F8FC2F064A136823F06A
:10894000807323F0010343F08073136008BD00BF00
:108950000010004074170040064B02280CBF042290
:108960000322C3F81025D3F8502642F00102C3F8C1
:108970005026704700100040014BC3F80C057047AB
:1089800000100040014BC3F808057047001000407C
:10899000074BC3F85405D3F8182522F00072C3F82A
:1089A0001825D3F8182542F00072C3F8182570472F
:1089B000001000400A4A0023C2F82C350123C2F8F7
:1089C0003035C378C2F82435437881781B0443EAF4
:1089D0000163017843EA0123C2F81C35704700BFE8
:1089E00000100040C2F34203022B10B50CBF4FF041
:1089F00080740024D307C0F108034FEA034300F05A
:108A00000F0040F4807003F470230B4A43EA000324
:108A100048BF44F480142343C2F81435D2F8180533
:108A2000064B0340C2F81835D2F8183543F44033EA
:108A30001943C2F8181510BD001000400000F8FEE0
:108A4000014BC3F80405704700100040014BC3F808
:108A5000040570470010004002280CBF2820292080
:108A60007047012070472920704702280CBF05205D
:108A70000A207047014B01221A6070470410004021
:108A8000014B01221A60704700100040074A4FF462
:108A90009063C2F8083501235360D360A2F5F03229
:108AA0000021C2F800121361704700BF00F00140BE
:108AB000044B0022C3F80021C3F80C21C3F8102195
:108AC000704700BF00100040034BD3F80001003096
:108AD00018BF0120704700BF00100040034BD3F8BF
:108AE0000C01003018BF0120704700BF001000408B
:108AF000034BD3F85005B0FA80F04009704700BF2F
:108B000000100040044B40F20312C3F83425C3F8B0
:108B10003805C3F83C15704700100040034BD3F8EC
:108B20000004003018BF0120704700BF0010004053
:108B300000487047640B002000487047680B002015
:108B4000044B03220021C3F8002202460846FFF727
:108B500047BE00BF00100040034B0321C3F80012C2
:108B600001460120FFF73CBE00100040054B0322E8
:108B7000C3F8002203F5F0334FF49062C3F80825E0
:108B8000704700BF00100040034AD2F8003243F49F
:108B90008873C2F80032704700100040014BD3F8D0
:108BA0004805704700100040024B0022C3F81C210A
:108BB000704700BF00100040034BD3F81C01003089
:108BC00018BF0120704700BF0010004030B50024DE
:108BD000A30003F1804303F580531568C3F80056E2
:108BE00001349588C3F82056082C02F10602EFD113
:108BF000024B40EA0120C3F8400630BD001000409F
:108C0000034AD2F8403623F0FF03C2F840367047DB
:108C100000100040024B0022C3F81421704700BF2F
:108C200000100040034BD3F81401003018BF01209E
:108C3000704700BF00100040014BD3F8100470478C
:108C400000100040054B4FF48022C3F8482303F581
:108C5000A0337F22C3F80825704700BF00B0004052
:108C6000034B044A1B7803F5A87342F823007047AE
:108C7000740C002000900040F8B5A2F57423314C2C
:108C8000DFF8D8C0A3F51073A34288BF02F1E872E1
:108C90002D4B2E4C82BF02F5D43201F1FF3102F58B
:108CA000A5720125B2FBF4F40026022204271D6000
:108CB000C3F8F864C3F80475C3F8FC24C3F834455A
:108CC000CCF848154FF48021CCF8441320490C3BD4
:108CD0000CF5A47CC1F818C5C1F81C35C1F80425F1
:108CE000FFF766FD1B4B1C4A1560C3F80465C3F80B
:108CF0001075C3F808651D60A3F5FD43743BC1F80A
:108D0000483503F500433433C1F84C25C1F85035DC
:108D100003F5AF33C433C1F85435A3F5AF33C03BCB
:108D2000C1F8583503F5AF33C833C1F85C354FF49B
:108D30001063C1F800384FF49053C1F8043820464E
:108D4000F8BD00BFBFBDF07F0C80004040420F0067
:108D500000F00140009000400C90004000B0004046
:108D6000044A01231360D3600C3202F6F4721360DC
:108D7000D3607047048000400C4B0D4AC3F8440593
:108D800003F5B833C3F8282502F5DE424032C3F8B4
:108D90002C2502F58072C3F83025A2F5E242343A60
:108DA000C3F834251822C3F804257047008000401A
:108DB000041100400B4B0C4AC3F8202502F5DE429B
:108DC0004032C3F82425A2F5DE423C3AC3F82825F8
:108DD00002F5DE424032C3F82C250C22C3F80425EC
:108DE000704700BF00F0014000110040014BD3F874
:108DF0004405704700800040014B1860704700BF79
:108E00006C0C0020014B1868704700BF6C0C0020F0
:108E1000014BD3F84005704700800040064B074ADD
:108E2000C3F8382502F5DE423C32C3F83C25202247
:108E3000C3F80425704700BF00F001400C1100404A
:108E4000014BD3F84805704700800040014BD3F830
:108E50004805704700800040164B70B5002402257D
:108E6000C3F80045144EC3F80055144D02290CBF39
:108E700029463146C3F80415C3F808051048C3F85D
:108E80000C05C3F810250F4AC3F814250E490F4AE4
:108E9000C3F80042C3F80441C3F80841C2F84015C2
:108EA00001F55F41C2F844154021C2F804150122C2
:108EB0001A6070BD00F000400100000101000101D6
:108EC000680B0020580A00200411004000F0014007
:108ED00010B50E4B00220224C3F80025C3F800454C
:108EE0000B4CC3F80445C3F80805C3F80C15094832
:108EF0000949C3F81005C3F814150121C3F800127D
:108F0000C3F80421C3F80821196010BD00F0004027
:108F100000000101680B0020580A00200C4B0222BF
:108F2000C3F80423D3F804216AB10222C3F808234A
:108F3000084A4FF40041C2F88011D3F80801B0FA92
:108F400080F04009704720BF40BF20BFEAE700BF64
:108F500000F0004000E100E0034BD3F800040030D3
:108F600018BF0120704700BF00F00040014BD3F84C
:108F70000004704700F00040044A0023C2F8283182
:108F800002F56042C2F80035704700BF0010004093
:108F9000084BD3F8280160B103F56043D3F8000112
:108FA00038B1D3F8040120B1D3F80801B0FA80F049
:108FB0004009704700100040012905D0404080F36F
:108FC00011884FF0040002DF18200AB1F8F7DEBC68
:108FD000F8F7ECBC39B1012908D0404080F3118882
:108FE0004FF0040002DF0B20F8F7F4BC1820FBE779
:108FF00088420AD018B94B1E584258417047012880
:1090000005D1B1FA81F04009704701207047002076
:1090100070470000084B39B101290AD0404080F365
:1090200011884FF0040002DF4FF40062C3F8002102
:1090300070474FF08072F9E700E100E0032805D99E
:10904000404080F311884FF0040002DF024B185CAF
:109050000028F5D0704700BF70B70000023810B488
:109060001C46032816D8DFE800F0020B1124032960
:1090700010D1134B00219C60002010BCF9F7D4BB29
:10908000042907D10F4B01219C60F5E7032907D084
:1090900004290AD0404080F311884FF0040002DF19
:1090A000094B00219C600120E7E7084B01219C60EF
:1090B000F9E70429EED1064B01219C600320DCE78F
:1090C000402B0020502B0020602B0020702B002014
:1090D000802B002001460020FFF714BB70470000E2
:1090E000014B03EB40107047842C00208279044B25
:1090F00003EB4213DB69C01A024BC01058437047A0
:10910000842C0020ABAAAAAA10B5094B827903EBE4
:1091100042130A689B695C6823689A4294BF0A609C
:109120000B60FFF7E3FFD4E9002302FB003010BD22
:10913000842C00202DE9F34105460191164601F0EB
:109140004DFC07464FF02003EFF3118883F311889D
:109150006B8A002B3DD02A8A9A422AD900212846C0
:1091600001F02CF9044620B388F31188019B002BF1
:109170003CD0731C012B06D901F030FCC01BB0425F
:1091800094BF361AB61BA3791E4F07EB4313324622
:109190009B691B6801A91B6820469847054620610A
:1091A00028BBA079214607EB401001F0E8F82C46D7
:1091B00018E06B8A5A1E6A8288F311882C8AE41A96
:1091C000EB69182202FB04340E4BED1A6D11A571E8
:1091D000CCE788F311883146284601F0EFF80446C1
:1091E0000028C3D1204602B0BDE8F08123610023EE
:1091F00023600122A280A381019A2369E281A360F6
:10920000F0E700BF842C002083695B680A46196878
:10921000FFF790BF836819440160704710B40A4695
:10922000146814B910BC01F0AFB8537943F00103CE
:1092300053712246F4E70000F8B5154D04460026A8
:1092400004B9F8BD23792768013BDBB22371002BF9
:10925000F7D1216959B163799B0707D4A37905EB4D
:10926000431320469B691B689B6898472661A07939
:10927000A66005EB401326605B691BB1204698474A
:109280003C46DDE7214605EB401001F078F8F7E7B2
:10929000842C0020037901330371704783880268AE
:1092A00019448180D018704730B4838804689D18B1
:1092B0008580E01830BCF8F72EBD83885B1A838068
:1092C0000368194401600846704708B50368012126
:1092D0001A78FFF7F2FF104608BD02688068101A7E
:1092E000704770B504680E4615464CB1A3681D4220
:1092F00004D063682A462146304698472468F4E73C
:1093000070BD00688068006841B9D0F8101521FA76
:1093100002F202F001021A6000207047D0F8102516
:10932000F9E700688068006851B9012101FA02F28A
:109330001BB1C0F8082500207047C0F80C25FAE7DB
:10934000C0F80435F7E78368186872B108605A6896
:10935000196002B959600020704710605868814256
:1093600008BF5A600DE0024600680028F3D088422A
:10937000F9D10868002AF0D15A681860914200D1EA
:10938000586000230B60E6E70021F8B50A460D4659
:109390000C4601268B0003F1804303F5C043D3F84C
:1093A000000168B1D3F81075D3F81005C3F8004177
:1093B000C0F3042306FA03F3B80454BF1A431D4351
:1093C00001310829E6D1084CA068836821461A407B
:1093D000FFF787FF6069826804F10C012A40BDE84D
:1093E000F840FFF77EBF00BF082C00200020704728
:1093F0000F4B30B51D68002325FA03F2D20710D5B4
:109400009A0002F1804202F5C042D2F81045C4F33E
:109410000424844205D1D2F81025C2F340328A4296
:1094200004D00133082BE7D16FF01203184630BD8A
:10943000B80C002070B514460D46C9B9036886689B
:109440009B6810461979FFF7D3FF00280FDBB2683D
:10945000012303FA04F4144300F14001064AB46006
:1094600003FA00F042F82150C2F80403284670BD08
:109470006FF02200FBE700BF0060004070B51446AB
:109480000D46B1B9036886689B6810461979FFF7E5
:10949000AFFF00280CDB0123B26803FA00F003FAE7
:1094A00004F4054B22EA0404B460C3F80803284618
:1094B00070BD6FF02200FBE7006000402DE9F04135
:1094C00006681446B268106819B16FF02200BDE852
:1094D000F08103F44071B1F5807FC3F30137C3F32A
:1094E000813203F440355BD0B1F5007F0CBF04211D
:1094F0000021B5F5803F02EB8702324F08BF0025FF
:1095000013F0010F57F8222004F5E07751D00C2911
:1095100048D10125A540C0F8085542F003020A438E
:1095200040F8272013F00200D1D0B26899061679CE
:10953000CBD55A0640D413F0040F0CBF4FF40035BE
:109540004FF48035204FD7F800804046F6F7B0FE44
:10955000082834D031462046FFF74AFF002809DAB0
:109560006FEA080292FAA2F0002AB0FA80F008BF6F
:109570004FF0FF300123834043EA08033B6023029E
:1095800003F4F853710343F0010301F4005100F5B3
:10959000A2700B430D4A2B4342F82030002096E77F
:1095A0000C21A6E7042902BF0125A540C0F80C55EF
:1095B000B3E70A432A43B3E74FF44035C2E76FF0FD
:1095C000040084E780B70000B80C00200060004071
:1095D00008B5002205210620F8F70AFA0620F8F758
:1095E000D5F9002008BD4FF0805210B514695369B9
:1095F0000144634399429ABFC043C00F002010BD8D
:10960000024AD2F80034002BFBD0704700E0014042
:109610002DE9F0474FF080521E4E057AD6F80485AA
:109620001769044615B1FAF705F805460223C6F88E
:109630000435FFF7E5FFDFF85C904FF0000A40F6D5
:109640007B362368C9F80835FFF7DAFF6368DB1B50
:10965000636023683B442360237A0AF1010A73B9EB
:109660006368002BEDD10B4BC3F80485FFF7C8FFEF
:109670006068003018BF01204042BDE8F087F9F76C
:10968000D9FF2946F9F7D8FFB0FBFAF31844B042E6
:10969000E6D9E8E700E0014070B58CB00DF12F018C
:1096A00004460DF12E00FEF74FFD9DF82E509DF85B
:1096B0002F60F9F7BFFF134A0592134A069400235F
:1096C00040F67B31CDE90331CDE90112CDE9073315
:1096D00000933246034603212846F9F74FFE30F047
:1096E000020308D145F6B311084801F05BF928B927
:1096F000A0680CB070BD6FF04700FAE76FF03B0058
:10970000F7E700BF1197000002DB8600D40C0020B1
:1097100070B58CB01D460646FEF750F90DF12F01CD
:109720000DF12E00FEF710FD134B9DF82E0006954F
:109730000024CDE9044310230093CDE907443346C8
:10974000CDE90244019422462146F9F717FE30F094
:1097500002030ED06FF04703AB609DF82F209DF8F9
:109760002E00009423462146F9F79CFE034801F0A1
:10977000F2F80CB070BD00BFD9970000D40C0020E7
:1097800070B50D462846194616461C46FFF72BFFB6
:1097900038B14CB1224629463046F8F7BCFA0020D1
:1097A00070BD6FF01500FBE72046F9E708B5012210
:1097B000064B43601146064801F0C4F8012200211F
:1097C000044801F0BFF8002008BD00BFECB700005E
:1097D000BC0C0020D40C002030B51D4685B0D3E968
:1097E00000309847044690B90DF10F010DF10E00BD
:1097F000FEF7AAFC9DF80F209DF80E00009423466A
:109800002146F9F74FFEAC60024801F0A4F805B01C
:1098100030BD00BFD40C0020F0B54FF0805387B0AE
:109820001D69B1FBF5F305FB13130F461646B2FB9A
:10983000F5F423B16FF01504204607B0F0BD05FB29
:109840001425002DF6D111463846FFF7CCFE00282E
:10985000F0D0002CF0D04FF0FF31104801F0A2F80A
:109860002846F9F76DFD88B101238DF8083003A86B
:109870000B4B0595CDE900760393CDF810D0FFF79B
:109880000BFF0446054801F066F8D5E78DF8140093
:1098900003A8CDE90376FFF7BBFEF2E7BC0C00207E
:1098A0001196000010B50A480C464FF0FF3101F048
:1098B00079F8084B4CB10022C3F80425FFF7A0FE4D
:1098C000034801F048F8002010BD0122F4E700BF72
:1098D000BC0C002000E00140F7B5057B044615B143
:1098E000F9F7A8FE0546676817F003006AD027F06D
:1098F000030702ABA268396843F8041DC0F10406EF
:10990000964228BF1646324618442168F8F703FAF3
:10991000FFF776FE019B3B60636833446360236816
:1099200033442360A3689E1B237BA660002B49D091
:10993000F9F780FE2946F9F77FFE40F67B33B3EB5B
:10994000400F3FD2FFF75CFE4FF0FF3003B0F0BD99
:10995000FFF756FE23681A6863681A606368043369
:109960006360236804332360A368043BA360237B04
:1099700001364BB1F9F75EFE2946F9F75DFEB0FB03
:10998000F6F31844B842DDD8A268032AE0D8AAB199
:10999000636821681B6802A840F8043DF8F7BBF92A
:1099A000FFF72EFE6368019A1A60D4E9012123684B
:1099B0000B440A44236000236260A360FFF720FE8B
:1099C0000020C3E7012640F67B37DDE770B50D4682
:1099D00088B01946284616461C46FFF704FE28B3F1
:1099E000DCB14FF0FF31134800F0DCFF0020F9F745
:1099F000A7FC04ABCDE90465069488B101228DF87B
:109A00001C20002203920C4A01A8CDE90123FFF794
:109A100043FE0446074800F09EFF204608B070BD94
:109A20008DF81C001846FFF757FFF2E76FF015049A
:109A3000F3E700BFBC0C0020D9980000034B186866
:109A400018B1D3F85C03C3F85C03704724210040CD
:109A5000024B8022C3F80423704700BF002000405F
:109A6000024B8022C3F80823704700BF002000404B
:109A7000024B1868003018BF012070471C210040BD
:109A8000024B0422C3F80423704700BF00200040AB
:109A9000024B0422C3F80823704700BF0020004097
:109AA000024B1868B0FA80F0400970471C21004052
:109AB000024B1868003018BF012070470821004091
:109AC000024B4FF40072C3F804237047002000409B
:109AD000024B4FF40072C3F8082370470020004087
:109AE00001207047014B1960704700BFEC0C00204B
:109AF000024B1B6803B11847704700BFEC0C0020F5
:109B00000A4BD3F80423120602D5094A126852B947
:109B1000D3F8040310F0040006D0064B1868003098
:109B200018BF012070470120704700BF002000408F
:109B30001C21004008210040F7B50023094C0A4FC2
:109B40001E46D8B2151A002D02DD256801330DB965
:109B500003B0F0BD266025680195019DD7F8185522
:109B60000D54EEE70821004000200040F7B5002327
:109B7000094C0A4F1E46D8B2151A002D02DD256881
:109B800001330DB903B0F0BD266025680195085C6E
:109B9000019DC7F81C05EEE71C2100400020004095
:109BA000074B00221A6082B01A680192019A054A96
:109BB000C2F81C151A68002AFCD0084602B070478B
:109BC0001C21004000200040084B1A6882B052B1AE
:109BD000002018601B680193019B054BD3F81835D2
:109BE0000B7002B070474FF0FF30FAE708210040D9
:109BF0000020004037B5204800F0A0F94368044633
:109C00005D68052201230021A847636805221D68BD
:109C1000002101232046A84763681D6800231946D8
:109C200003222046A847154B0322C3F8142505221A
:109C3000C3F80C250024124AC3F86C45C3F8242548
:109C40000422C3F800250F4A146012680192019A99
:109C50000D4A146012680092009A0C4A01211160AA
:109C6000022019602246F7F7C3FE0220F7F78EFEA6
:109C7000204603B030BD00BFD9B100000020004035
:109C800000E0D7011C2100400821004008200040CE
:109C90002DE9F0418378C4781E1DA3420A4406448E
:109CA0001FD8E41AE4B2A1423EBF641AE7B20C46E0
:109CB0002344A1EB040128BF0027DBB2C9B234441E
:109CC000A64209D183704378BB4282BF204B012258
:109CD0001A600846BDE8F08116F8015B02F8015DE4
:109CE000EEE70578ED1AEDB2A9423FBF671AED190C
:109CF000EFB20D4638BF5B18A1EB050132BFDBB2F6
:109D000027460023C9B2944606EB050E764519D1C5
:109D1000521B0029D6D0002CD4D08C428ABF0B46CF
:109D20002346641A00F10406A1EB03018CBFE7B2DD
:109D30000027C9B2F418A642C4D016F8015B02F895
:109D4000015DF8E716F8018B0CF8018DDEE700BF26
:109D500000D0004030B5D0B1C27805788478531C6B
:109D6000DBB29D4208BF00239C4210D061B10A497A
:109D70000244D1F808151171C3700133DBB29D4262
:109D800008BF00239C4205D06FF00F0030BD6FF07C
:109D90003600FBE70020F9E700D0004070B584688A
:109DA00001221146204600F0CDFD04F118000122E9
:109DB000002100F0C7FD042384F831300C23002576
:109DC00084F83D300521114B84F830100D2684F8BD
:109DD000335084F8325084F83C6084F83F5084F863
:109DE0003E50D3F8042542F00102C3F804250122B5
:109DF000C3F800513046C3F804231A602A46F7F727
:109E0000F7FD3046F7F7C2FD284670BD00D0004090
:109E1000DB0770B5144617D480680A463C30E1B2BF
:109E2000FFF736FF70BDC2F800511060D2F8006134
:109E3000002EFBD0013B9BB2D2F80865CE54002B1C
:109E4000F1D150602046EDE713460120014A00257C
:109E5000F5E700BF00D0004070B5134CD4F80031D6
:109E60005BB18568012105F13C00FFF773FF10F13C
:109E7000100F03D10023C4F8003170BD373014BF78
:109E80000021012105F13000FFF764FF064605F1CE
:109E9000180000F060FD00231036C4F800311EBF2A
:109EA000024B01221A60E8E700D0004004D00040D5
:109EB0002DE9F84385680F46144605F1180814B9D2
:109EC0002046BDE8F883FF2C234628BFFF23E41A71
:109ED000DEB2A4B205F130094FF0FF31284600F0A0
:109EE00061FD31463A464846FFF7D2FE064628460F
:109EF00000F031FD002EE2D04FF0FF31404600F07F
:109F000051FDE9E7134602480A461946FFF7C0BE6D
:109F10002C0D002038B5084B53F82040013053F881
:109F200020502046854204F10C0400D838BD54F876
:109F30000C3C5B689847F4E760B80000104B70B5C4
:109F4000104C05461E469C4204D10E4CB44209D129
:109F5000002412E062681AB122681268AA420CD08A
:109F60000C34F0E763680BB90C34EFE7236828463C
:109F70001968F7F7B3FE0028F6D1204670BD00BF80
:109F8000442C00209C2B0020431C03D0034B1B6857
:109F9000834201DCF7F7BEBA704700BF902B002068
:109FA0000F4D80B50F4F05F114064FF02002EFF36F
:109FB000118382F311886B69B3420AD04BB11C69DB
:109FC000631C08D03B68A34205DDEC61F7F766FD32
:109FD000EBE74FF0FF342046F7F782FAF5E700BFD2
:109FE000940F0020902B00200248034A0021121AEF
:109FF000F7F7BEBE00000020501000200248034AC0
:10A000000349121AF7F787BE48290020C42C002004
:10A01000B4B8000008B50220FFF77CFF0748F6F748
:10A020005BFF0320FFF776FF00F0BCFEF6F794FB22
:10A03000034A137A23F00103137208BD7CB80000B1
:10A04000B00D002080B586B006AFF7F7EBFA2E4BC7
:10A0500083F308882D4B2E4D2E4E0024E02283F8EA
:10A060002220DC771C765C769C765A6A42F4E022E9
:10A070005A62F7F783FCF7F70BFD2046FFF74AFF1C
:10A080000120FFF747FF00F0F3FB012335624FF497
:10A090008062CDE90343CDE9014400941E4B1F4982
:10A0A000284600F027FE6B7A23F0040213F01B0F02
:10A0B0006A72344605D16B6A013302D1284600F03A
:10A0C000D3FA174E17490F230122CDE9033200239B
:10A0D000CDE9013300934FF4A072134B304600F0EA
:10A0E00009FE737AE66023F0040373720F4BA560D8
:10A0F000C4E90533084A0E4B0E4C83F3098800214E
:10A1000081F31188104620474825002000ED00E02B
:10A11000B00D0020940F002015A0000008180020AA
:10A12000400D0020081C0020A19F0000A80F002067
:10A13000081C0020E507000038B5074C074DAC426D
:10A1400001D3002038BD04F114032046C4E90533CF
:10A15000F6F783FB1C34F2E7442C0020442C00204B
:10A160002DE9F04F1D1E85B007460C4692464CDD8A
:10A1700000F03EFC05F109030A22B3FBF2F310EBF9
:10A180000308234B234EFB1A9B105E43F6B207F1E4
:10A19000140B009403AB02AA51463846F6F7A6FB0F
:10A1A00010F10B0F0BD1009403AB02AA51463846B5
:10A1B000F6F79CFB10F10B0F08BF6FF00B006379F3
:10A1C000029A267162F3030363716368039A62F370
:10A1D0001F336360B0B1ADB110F10C0F12D14FF06D
:10A1E0002003EFF3118083F311882A46594600F0CB
:10A1F000E9FA6B1CCDD000F0FBFBB8EB0005C8D52D
:10A200006FF00A0005B0BDE8F08F4FF00008B8E726
:10A21000442C0020B76DDBB670B504780268417835
:10A22000134EC4EBC404A400120B01F00F0130194B
:10A23000F6F710FC4FF02003EFF3118583F311883C
:10A2400004F11400304400F003FB68B1EFF3058320
:10A250000D2B09D81BB1074B5B681B0504D528469D
:10A26000BDE8704000F0A8B985F3118870BD00BF4B
:10A27000442C002000ED00E013B504240A1904D298
:10A2800000236946FFF76CFF10B1002002B010BD3B
:10A29000224601A90098F7F73EFD00980430F5E743
:10A2A00010B10438FFF7B8BF70470000034B9B683C
:10A2B0000146586E08B1FFF7DFBF7047940F0020CA
:10A2C000F8B504460E4617464FF02002EFF311850D
:10A2D00082F311889BB10820FFF7E8FF002832D0F5
:10A2E000012347600360036803F0030256B9236843
:10A2F00013430360636820606BB960600BE03B60F0
:10A300003846F0E7336833F0030314D10260626823
:10A310005AB9C4E90000042104F1080000F0E6FE87
:10A32000284600F049F90020F8BD136803F0030344
:10A3300003431360E1E713430360336803F003034F
:10A3400018433060E7E76FF00B00EDE710B5044607
:10A3500030B10268930703D0446809B1FFF7A0FF4A
:10A36000204610BD0023C0E9003300F10803C0E916
:10A37000023370470A4600234168FFF7A1BF00235C
:10A380000A461946FFF79CBF38B54FF02003EFF39C
:10A39000118583F31188436853B901604260042139
:10A3A000083000F0A3FE2846BDE8384000F004B9AC
:10A3B0001C6804F0030421431960EFE72DE9F04124
:10A3C000044686B00D464FF02003EFF3118783F368
:10A3D0001188026882B11368416823F003038A423E
:10A3E000036008BF436001211046FFF7AFFF87F30A
:10A3F000118806B0BDE8F08119B987F311880020F3
:10A40000F7E787F31188042103460DEB010000F004
:10A41000D6FD6A1C02D000F0E1FA064600279DF83E
:10A420001130EA1B6FF30713012101A88DF81130D9
:10A4300000F0D8FD08B10B30E1D14FF02003EFF36D
:10A44000118883F31188206838B10368626823F0AB
:10A4500003039042236008BF63600121FFF776FF8A
:10A4600088F311880028C4D16B1CD8D000F0B6FA4C
:10A47000871BBD42D3DAC2E7D0E900231A60026825
:10A48000536070470146006908B5431C0ED0084B65
:10A490009B6999421FBF0A681369C018106108467A
:10A4A000FFF7EAFF4FF0FF330B61002008BD00BF4C
:10A4B000940F00204FF02003EFF3118083F31188F5
:10A4C000704700000D4B1A4652F8241F914200D0ED
:10A4D00001B9D96870B99A6862B1507AC00609D1D9
:10A4E000506A013006D150897F2803D9044800689A
:10A4F000824201D1196270471A627047940F00209E
:10A5000078B8000090F90A0091F90A309842ACBF7F
:10A51000002001207047000010B50146FFF7CAFF78
:10A520004B7A5A0604460DD50846FFF7A5FF4B7A2D
:10A5300023F040034B72054B9868431A5842584128
:10A54000FFF7C0FF84F3118810BD00BF940F0020F7
:10A5500008B50246FFF7AEFF13689A4208BF002312
:10A5600080F31188184608BD10B50146FFF7A2FF19
:10A5700004460846FFF780FF4B7A23F002034B7234
:10A5800084F3118810BD10B50021FFF7E1FF0446E8
:10A5900028B1FFF7E9FF04F11400FFF773FF20462D
:10A5A00010BD10B50446FFF7DFFF04F11400BDE84D
:10A5B0001040FFF767BF0000EFF305830D2B0ED8A7
:10A5C0001BB1094B5B681B0509D5084B9A681B6AD0
:10A5D0009A4204D0064B00221A60F7F72FB880F396
:10A5E00011880020704700BF00ED00E0940F0020AC
:10A5F000C40F002010B5FFF75DFF0A4B9A68D37AAD
:10A6000001330446D3720120FFF75CFF84F3118805
:10A610004FF02003EFF3118083F31188BDE8104061
:10A62000FFF7CABF940F00200368984210B513D0FB
:10A6300093B191F90A2093F90A40944206DD5A68D1
:10A64000C1E900325A681160596010BD4468A342E4
:10A6500002D01B68002BEED143684B604368086052
:10A6600019604160F1E7000038B50446FFF722FFAA
:10A67000214605460648FFF7D7FF637A43F04003BB
:10A6800063720020FFF71EFF85F3118838BD00BFFD
:10A69000B80F0020427AD20604D1436A013301D1B7
:10A6A000FFF7E2BF7047000070B50B6104461D461E
:10A6B000C1E902020BBB4FF02003EFF3118683F3D5
:10A6C00011884FF0FF330B6170B1CB6813B1FFF706
:10A6D0004BFF2562637A23F0040363722046FFF781
:10A6E000D9FF86F3118870BD86F311884B69002B62
:10A6F000F9D00846BDE870401847114AD2E905363E
:10A7000002F114008342054613D093B108691C6915
:10A71000A04208DC5A68201A1861C1E900325A6860
:10A7200011605960DFE7001BB342086101D01B686C
:10A73000EBE7C1E90056936919609161D3E700BF67
:10A74000940F002038B50446FFF7B4FE05462046B6
:10A75000FFF792FE21460648FFF766FF637A43F053
:10A76000400363720020FFF7ADFE85F3118838BD0A
:10A77000B80F0020F8B5054614460E46FFF7CCFE8C
:10A780006B7A43F002036B72631C12D04FF020030C
:10A79000EFF3118783F311880A2309343246B4FB9F
:10A7A000F3F305F1140101332846FFF77DFF87F32A
:10A7B00011882EB129463046BDE8F840FFF734BF76
:10A7C000F8BD000010B5064B04469868FFF7D2FFAD
:10A7D000044B00222046BDE810401A60F6F72EBF59
:10A7E000940F0020C40F0020134B1B68002B10B5E2
:10A7F00002461FDD43897F2B1CD8104B90F90A10AD
:10A800001B68994216DBFFF755FE0D4951F8243FAE
:10A810008B4204460AD05BB192F90A0093F90A30E0
:10A82000C31A5842584184F3118810BD0020FAE73A
:10A830001846F8E70020F8E7200E0020240E00203C
:10A84000940F0020014B00221A607047C40F0020B3
:10A8500038B5054600202C68A54200D004B938BDA3
:10A860002046FFF79EFE2046FFF714FF0120F2E787
:10A87000024B03F12402C3E909227047940F002020
:10A8800038B5144C144BA2681B689A420FD0FFF7DE
:10A8900011FE0546A068FFF7EFFDA16804F1240052
:10A8A000FFF7C2FE0120FFF70DFE85F31188A268B5
:10A8B000236A9A420CD04FF02003EFF3118083F308
:10A8C0001188064B00221A60BDE83840F6F7B6BE84
:10A8D00038BD00BF940F002078B80000C40F0020DE
:10A8E00037B520B903B0BDE83040FFF7C9BF0A2330
:10A8F0000930B0FBF3F0013001904FF02003EFF38B
:10A90000118583F311880A4CA068FFF705FEA06843
:10A91000019B00F114010022FFF7C6FE054B002247
:10A9200028461A6003B0BDE83040F6F787BE00BF86
:10A93000940F0020C40F0020014B9868704700BF9F
:10A94000940F002000F11003C0E90212C0E90000DA
:10A95000C0E90433704770B504464FF02003EFF3AD
:10A96000118683F31188FFF70EFE054670B1437A16
:10A97000DB0604D1436A013301D1FFF775FE0023E2
:10A98000EB663046BDE87040FFF716BED4E90232F0
:10A990009A4218BF0133A360022104F1100000F0B5
:10A9A000A5FBEEE710B40A4604464FF02003EFF390
:10A9B000118083F31188A36833B1013BA36080F356
:10A9C0001188002010BC704721B980F311886FF006
:10A9D0000F00F7E7214610BCFFF7F4BE034BD3E9A5
:10A9E00000230A231046A0FB03017047C80F002074
:10A9F0004FF02002EFF3118382F31188024AD2E96B
:10AA0000000183F311887047C80F00202DE9F04F33
:10AA1000074685B04FF02003EFF3118083F31188D0
:10AA20006149D1E90045E21945EBE773C1E900232B
:10AA300080F3118802AECDE902664FF02003EFF3F8
:10AA4000118083F31188594C2146024651F8143F76
:10AA50008B4200D0FBB980F31188A068FFF7C4FED9
:10AA6000B0B1534A11680A2307FB0317514B176013
:10AA70001B689F420CDB002313604FF02003EFF3B1
:10AA8000118583F31188A068FFF75CFE85F31188B8
:10AA900005B0BDE8F08F484D0195012129604FF0C8
:10AAA000000C39466FF0010E18698842AABFA0EB6E
:10AAB0000108C3F810C0C3F81080091AA0691D6905
:10AAC000984214BF18680020D5B9D3E90059C9F8D5
:10AAD00000501D68C5F80490029DC3E90056029D10
:10AAE00002936B60C3F810E082F311884FF02003EB
:10AAF000EFF3118283F3118803460028D4D101E0DB
:10AB00000029F1DC82F311880298B04203D1019A46
:10AB100000231360A1E70028F9D00668039B4FF0DB
:10AB2000FF39984208BF00264FF0000AD0E9002301
:10AB30001A600268D0F808B053604FF02003EFF3BA
:10AB4000118883F31188C0F81090BBF1000F1FD05B
:10AB5000C36823B15846FFF707FDCBF820A09BF848
:10AB6000093023F0040213F01B0F8BF8092006D1E3
:10AB7000DBF82430013302D15846FFF775FD88F326
:10AB80001188002EC3D0039BB34208D1002307E0F5
:10AB900088F311884369002BF3D09847F1E73368B5
:10ABA00030461E46C2E700BFC80F0020940F0020A9
:10ABB000C40F0020200E0020C00F002008B54FF465
:10ABC00080624FF0FF330349034800F061F9002031
:10ABD00008BD00BF48250020D00F002003695A1C83
:10ABE00010D009490268896988421EBF11695B1843
:10ABF000136143681A60026853604FF0FF330361CA
:10AC00000020704718467047940F0020427AD20601
:10AC100004D1436A013301D1FFF726BD704700001C
:10AC2000F0B54FF02003EFF3118683F31188184A33
:10AC3000C0610A230931B1FBF3F1013141621146D0
:10AC40000023036251F8143F8B4200F1140518D021
:10AC5000BBB1D2F818C0446A1F69BC420ADC5A680A
:10AC60003C1B1C61C0E905325A6815605D6086F3C3
:10AC70001188F0BDE41B6345446202D01B68002BC1
:10AC8000E9D193698361936941611D609561EEE744
:10AC9000940F0020EFF305800D2807D838B1044B3E
:10ACA000586880F40060C0F3C020704701207047EE
:10ACB00000ED00E0024B9B68187A00F0010070473D
:10ACC000940F002010B54FF02003EFF3118483F3AD
:10ACD0001188437A590702D484F3118810BD23F0F8
:10ACE00004034372FFF792FF2046BDE81040FFF7D0
:10ACF00063BC000030B587B004460E9D04950D9DE1
:10AD000003950C9D02950B9D01950A9D0095F6F704
:10AD100097FE044B9B6813B9636607B030BD5B6E4A
:10AD2000FAE700BF940F002070B586B0DDE90E652C
:10AD300004960D9E03960C9E02960B9E01960A9E0B
:10AD400000960446FFF7D6FF6B1C03D02DB92046B2
:10AD5000FFF7B8FF204606B070BD29462046FFF732
:10AD60005FFFF7E7436D10B5044603B19847637A78
:10AD7000DA060AD1626A013207D12046FFF7CCFB1E
:10AD8000637A43F00803637210BD9B0702D5204627
:10AD9000FFF7EAFB636A0133F2D004F11400FFF716
:10ADA0001DFFEDE7F0B5214F214D87B03E46BD4276
:10ADB00005F12C0414D31F4B9A68D37A013BD3724C
:10ADC0004FF02003EFF3118583F31188184CB44240
:10ADD00020D385F3118807B0BDE8F040FFF70ABC27
:10ADE00054F80C3C049354F8103C039354F8143C6E
:10ADF000029354F8183C019354F81C3C009354E916
:10AE0000092354E90B01FFF775FF54F82C3C1D652D
:10AE10002546CCE7616A4B1C03D0206819B9FFF7BF
:10AE200051FF2C34D3E7FFF7FBFEFAE7442C002058
:10AE3000442C0020940F00200372427200234FF034
:10AE4000FF328172C372C0E90832C3618362704706
:10AE500010B504464FF0FF312046FFF7AFFA034626
:10AE60000028F7D008334268BFF35B8F53E8001F18
:10AE700021F0010C43E800CEBEF1000FF6D1BFF384
:10AE80005B8FCB0700D59047FFF7FAFCE2E70000A5
:10AE9000F0B587B004461F460D461646FFF762FA26
:10AEA0000020CDE90400CDE90207CDE90040044BC4
:10AEB0003246294604F11000FFF736FF07B0F0BD17
:10AEC00051AE0000836870B505460E46D3B100222E
:10AED0001C685A60637A9A0714D5636A02331AD0E1
:10AEE0002046FFF75EFB002E0CBF6FF0030300232C
:10AEF000E366637ADB0605D1636A013302D120463B
:10AF0000FFF7B2FB6B7B46EA1316002066F30713CC
:10AF1000A8606B7370BD6FF00A00FBE7F8B51746C9
:10AF2000D0E90023904204460D4606D163686B6069
:10AF300063682C601D60656019E0002BF6D09B688B
:10AF400039681868FFF7DEFA0028EFD12668B442A6
:10AF5000ECD0002EEAD0B36838681968FFF7D2FA4F
:10AF600030B17368C5E9006373681D607560F8BD32
:10AF700063689E42DAD03668EBE7142330B503FBF2
:10AF800001000024002900DA30BD437B846003F017
:10AF90000F03022B03D0042B01D0012B04D1D0E9E5
:10AFA00000531D6005686B6082F311884FF0200329
:10AFB000EFF3118283F3118801391438E2E730B5D9
:10AFC000447B036161F30304817B62F300018173BD
:10AFD000C289002565F3071465F34F028560447349
:10AFE000C28130BD2DE9F04F3F4B85B09B68009387
:10AFF0000026012307468A469046019304464FF0F7
:10B00000FF35B146564510DB4FF02003EFF31186B4
:10B0100083F31188019C002C49D1324629463846D9
:10B02000FFF7ABFF86F311884AE04FF02003EFF300
:10B03000118B83F31188627B02F00F03022B03D084
:10B04000042B04D0012B13D12169896801E0216907
:10B05000096869B143EA121363F307126273C4F813
:10B060000890CDF804908BF3118801361434C9E7A9
:10B07000B8F1000FF7D0019A002AF4D0022B07D0C4
:10B08000042B0FD0012B09D16A462146206903E029
:10B0900020696A4621461030FFF740FFC4F808D007
:10B0A0000135E0E720696A4621460830F4E70023CD
:10B0B0000193B8F1000F07D186F311886FF00A04ED
:10B0C000204605B0BDE8F08F02A942463046CDE9E2
:10B0D0000211FFF777FB04464FF02003EFF31186D0
:10B0E00083F3118899E700BF940F0020036898420A
:10B0F00007D0D3E900021060186842601846FFF7D5
:06B10000E1BE704770473C
:08B10800D051FF7F010000009F
:10B1100075B30000A90700000000000075B300002F
:10B12000911100000000000068B200000D12000044
:10B130000000000073B200000D12000000000000CB
:10B140007EB20000411500000000000075B3000051
:10B15000751C00000000000075B30000E936000017
:10B1600000000000E0B10000ED930000C8B700004F
:10B17000D9B10000D1950000C0B7000000B80000B0
:10B18000AD97000000000000E7B10000F59B000053
:10B190000000000044B200009D9D0000000000007F
:10B1A00075B3000039A100000000000075B3000075
:08B1B000BDAB0000000000002F
:10B1B80000FFFFFFFFFFFF0C0802170D0101020946
:10B1C8000901010602091818030101090903030509
:10B1D800034750494F5F30004750494F5F31005592
:10B1E8004152545F30004E52463532383430206276
:10B1F8006F61726420636F6E74726F6C2073746118
:10B20800746963616C6C7920636F6E6669677572C7
:10B2180065642E20444B20557074696D65206973F0
:10B22800202564207365636F6E64730A00464C4181
:10B2380053485F30005352414D5F3000454E5452E1
:10B248004F50595F300000007113000000000000EB
:10B258000000000025120000AD11000000000000F1
:10B26800636C6B5F6B333273726300636C6B5F6D1F
:10B278003136737263007379735F636C6F636B004D
:10B288002A2A2A2A2A20425553204641554C54201E
:10B298002A2A2A2A2A0A00202050726563697365BF
:10B2A800206461746120627573206572726F720A1E
:10B2B800002020496D70726563697365206461744C
:10B2C8006120627573206572726F720A00202049CE
:10B2D8006E737472756374696F6E2062757320651E
:10B2E80072726F720A0052657365727665642045E2
:10B2F8007863657074696F6E202800537075726981
:10B308006F757320696E7465727275707420284940
:10B31800525120002A2A2A2A2A20484152442046EB
:10B3280041554C54202A2A2A2A2A0A0020204275EC
:10B3380073206661756C74206F6E20766563746F18
:10B3480072207461626C6520726561640A00202055
:10B358004661756C7420657363616C6174696F6EA6
:10B3680020287365652062656C6F77290A002A2A90
:10B378002A2A2A204465627567206D6F6E69746F8A
:10B388007220657863657074696F6E20286E6F74BB
:10B3980020696D706C656D656E74656429202A2A54
:10B3A8002A2A2A0A002A2A2A2A2A202573202564DA
:10B3B80029202A2A2A2A2A0A002020457865637526
:10B3C80074696E6720746872656164204944202836
:10B3D800746872656164293A2025700A20204661E4
:10B3E800756C74696E6720696E73747275637469BD
:10B3F8006F6E20616464726573733A20203078251B
:10B40800780A002A2A2A2A2A204D505520464155D2
:10B418004C54202A2A2A2A2A0A00202053746163BD
:10B428006B696E67206572726F720A002020556E14
:10B43800737461636B696E67206572726F720A005C
:10B4480020204461746120416363657373205669E9
:10B458006F6C6174696F6E0A0020204164647265C4
:10B4680073733A20307825780A002020496E737467
:10B4780072756374696F6E204163636573732056D8
:10B48800696F6C6174696F6E0A002020466C6F6189
:10B4980074696E672D706F696E74206C617A79209B
:10B4A800737461746520707265736572766174690E
:10B4B8006F6E206572726F720A002A2A2A2A2A2061
:10B4C8005553414745204641554C54202A2A2A2A9B
:10B4D8002A0A0020204469766973696F6E206279B0
:10B4E800207A65726F0A002020556E616C69676E5C
:10B4F8006564206D656D6F72792061636365737330
:10B508000A0020204E6F20636F70726F636573733B
:10B518006F7220696E737472756374696F6E730AE3
:10B52800002020496C6C6567616C206C6F61642039
:10B538006F66204558435F52455455524E20696EF8
:10B54800746F2050430A002020496C6C6567616C59
:10B5580020757365206F66207468652045505352C6
:10B568000A002020417474656D707420746F206522
:10B5780078656375746520756E646566696E656463
:10B5880020696E737472756374696F6E0A002A2A73
:10B598002A2A204B65726E656C20416C6C6F636162
:10B5A80074696F6E204661696C75726521202A2A5C
:10B5B8002A2A0A002A2A2A2A2A204B65726E656CD2
:10B5C800204F4F505321202A2A2A2A2A0A002A2AA1
:10B5D8002A2A2A204B65726E656C2050616E696359
:10B5E80021202A2A2A2A2A0A002A2A2A2A20556EAB
:10B5F8006B6E6F776E20466174616C204572726F56
:10B608007220256421202A2A2A2A0A004375727288
:10B61800656E7420746872656164204944203D2019
:10B6280025700A4661756C74696E6720696E73745B
:10B6380072756374696F6E206164647265737320D8
:10B648003D20307825780A004953520065737365A8
:10B658006E7469616C207468726561640046617417
:10B66800616C206661756C7420696E2025732120D9
:10B678005370696E6E696E672E2E2E0A00466174CD
:10B68800616C206661756C7420696E2074687265DF
:10B698006164202570212041626F7274696E672E83
:10B6A8000A00000074B70000BCB6000074B70000C0
:10B6B800C4B600004C000000801000204C000000C0
:10B6C80060110020E0B6000000000000000000004B
:10B6D800E5370000F9360000436F6E74726F6C6CCA
:10B6E8006572007075626C69630072616E646F6D7B
:10B6F800007075626C69632069640072616E646FC2
:10B708006D20696400307825303278002530325851
:10B718003A253032583A253032583A253032583A9C
:10B72800253032583A253032582028257329005AB6
:10B738006570687972204F532076312E31322E3958
:10B7480039204465632020352032303138203232A8
:10B758003A30383A30310000F401FA0096006400BB
:10B768004B0032001E00140003040005099100007C
:10B7780000000000DD900000000000000002000052
:10B7880000000000000600000001000000030000A7
:10B79800000000000007000000000000000000009A
:10B7A8000000000000000000000400000005000088
:10B7B8000000000000000000000000500000000031
:10B7C8000003005001000000BD9400002393000016
:10B7D8000393000047930000359400007D94000017
:10B7E8000000000081970000CD9900001998000022
:10B7F800A5980000010000004E52465F464C415398
:10B80800485F4452565F4E414D450000C99B0000B9
:10B81800A19B00003D9A00006D9B0000399B000031
:10B82800519A0000619A0000719A0000819A000004
:10B83800919A0000A19A0000B19A0000C19A0000F4
:10B84800D19A0000019B0000E19A0000E59A0000EF
:10B85800B19E0000119E00009C2B0020FC2B0020B4
:10B86800082C0020442C0020442C0020F5FFFFFF6A
:10B87800400D00202A2A2A2A2A20426F6F74696EF6
:10B8880067205A6570687972204F532076312E31BF
:10B89800322E302D3331332D67646165663363632F
:0CB8A8003562202A2A2A2A2A0A00000001
:10B8B40002000000502900200000000035B2000002
:10B8C40026000802000000203DB2000022000811FA
:10B8D4006D0B00000090D0034B110000000000002D
:10B8E4000000000000000000000000000000000054
:10B8F4000000000000000000000000000000000044
:10B904000000000000000000000000000000000033
:10B914000000000000000000000000000000000023
:10B924000000000000000000000000000000000013
:10B934000000000000000000000000000000000003
:10B944000000000000000000CD2300000000000003
:10B9540000000000000000000000000000000000E3
:10B964000000000000000000002A0020002A00203F
:10B974000100000001000000102A0020102A00200D
:10B98400000000000000000000000000242A002045
:10B99400242A002000000000FFFFFFFFFF1F00001B
:10B9A4001F0000000000000000000000140400203C
:10B9B40000000000494F000000000000D4030020F4
:10B9C400010000000149000000000000DC03002029
:10B9D400000000003149000000000000A003002026
:10B9E400000000003149000000000000A80300200E
:10B9F40000000000314900000000000004040020A1
:10BA0400000000003949000000000000B0030020DD
:10BA1400000000003949000000000000B8030020C5
:10BA24000000000039490000000000001C04002050
:10BA3400000000000000000000000000E4030020FB
:10BA4400000000002954000000000000EC03002066
:10BA5400000000002954000000000000F40300204E
:10BA6400000000003954000000000000FC03002026
:10BA7400000000003954000000000000C003002052
:10BA8400000000003954000000000000C80300203A
:10BA94000000000039540000000000000C040020E5
:10BAA40000000000F974000000000000780C002081
:10BAB40000000000B12A000000000000800C0020FB
:10BAC40000000000592B000000000000880C00203A
:10BAD40000000000B12A000000000000900C0020CB
:10BAE40000000000592B000000000000980C00200A
:10BAF40000000000592B00000300000001000000BA
:04BB040047010000F5
:10BB080010B100000000000000000000A0B100001B
:10BB180000000000000000004CB100000000000020
:10BB28000000000028B1000050B200000000000032
:10BB380034B100005CB200000000000088B10000D1
:10BB480014B800000000000094B1000058B80000CC
:10BB5800F00C00201CB100000000000000000000F4
:10BB680040B10000000000000000000070B10000BB
:10BB7800D0B70000A00C002064B10000D0B70000CE
:10BB8800AC0C0020ACB10000000000000000000078
:10BB980058B1000000000000000000007CB1000067
:08BBA800000000000000000095
:10BBB000442C0020442C002000000000FFFFFFFF69
:10BBC000542C0020542C00205C2C00205C2C0020E5
:10BBD00000000000FFFFFFFF6C2C00206C2C0020F9
:10BBE00000000000000000007C2C00207C2C0020C5
:10BBF00000000000000000008C2C00208C2C002095
:10BC00000200020000000000ACB60000501000204E
:10BC10000000000000000000AC2C0020AC2C002034
:10BC20000300030000000000B4B60000181100205B
:0400000300001C11CC
:00000001FF
